:020000040800F2
:100000000080002089BC0008ABBD00080D930008EB
:1000100000000000000000000000000000000000E0
:10002000000000000000000000000000ADBD00085E
:100030000000000000000000AFBD00082D93000884
:10004000BDBC0008BFBC0008C1BC0008C3BC0008A0
:10005000C5BC0008C7BC0008C9BC0008D59600088C
:10006000CDBC000871930008D1BC0008D3BC0008C7
:10007000D5BC0008D7BC0008D9BC0008DBBC000810
:10008000DDBC0008DFBC0008E1BC0008E3BC0008E0
:10009000E5BC000801970008E9BC0008EBBC0008BB
:1000A000EDBC0008EFBC0008F1BC00085D9400083E
:1000B000F5BC0008F7BC0008F9BC0008FBBC000850
:1000C000EDAF16204A62304029BD56B31544E9BF52
:1000D00077900D9CFE0B88C07E2615FA83807340B6
:0800E0000FCE674B80D541C033
:1000E800000000000000244000000000000059400B
:1000F800000000000088C3400000000084D797413A
:100108000080E03779C34143176E05B5B5B893460B
:10011800F5F93FE9034F384D321D30F94877825AD7
:080128003CBF737FDD4F15752C
:1001300001000000000000000A00000000000000B4
:100140006400000000000000E80300000000000060
:100150001027000000000000A08601000000000041
:1001600040420F0000000000809698000000000050
:1001700000E1F5050000000000CA9A3B0000000005
:1001800000E40B540200000000E87648170000006D
:100190000010A5D4E800000000A0724E180900006D
:1001A00000407A10F35A00000080C6A47E8D030040
:1001B0000000C16FF286230000008A5D784563016C
:1001C000000064A7B3B6E00D0000E8890423C78AE5
:1001D00010B5816A8A6D50231A428A6D05D0D20605
:1001E00002D4096D496B884710BD012043021A43B0
:1001F0008A650A68D3681B059B0F02D01049086006
:1002000010BD8B7E002BF9D113681B07F6D59368C0
:100210005B0709D4583153680C24A3435360FF2370
:1002200002330A689A4305E08A6D202313438B65E5
:10023000CA6D5C3102430A600149086010BDC046C6
:04024000080F002083
:10024400F0B58BB000240A9454259A4E715D0129AF
:1002540000D111E10127775531688A68520714D417
:10026400336942680992022A944A13D104273B4312
:1002740093426AD1904AD3430268D04318438B6AAD
:1002840003408B62002A64D4F5E0B06D2021014361
:10029400B165F0E0089104210B439342864B67D18A
:1002A40007683B4008998A6A1A438A623A024B6992
:1002B400934380681040824A02401A434A61002FE7
:1002C40000D4D8E001237F483A4607680720800518
:1002D4003946099001407C480792824200D08EE062
:1002E400D8053A46024000D089E0764F3A68099B27
:1002F4009A431143014339607648006876490AF00D
:100304006FFB0C2141430C310A910A98002800D15B
:10031400B1E00A98401E0A900A98002800D1AAE089
:100324000A98401E0A900A98002800D1A3E00A986F
:10033400401E0A900A98002800D19CE00A98401EAA
:100344000A900A980028E4D195E00268002A00D4B3
:1003540091E05C4801685D4B9A4200D182E05C4BBD
:100364009A427CD0584B9A4200D084E005227AE02D
:10037400029106941F26099A16400F2201920596AF
:10038400B2404C4E346E03929443049402681A4271
:10039400079249D0D207069C2346089948D1079A68
:1003A40092073B4644D4079B5A0767D41A0767D47D
:1003B400DA06029B3CD4079B9A0663D45A0663D49C
:1003C4001A0663D4DA0563D49A0563D45A0563D450
:1003D4001A0563D4DA0463D49A0463D45A0463D444
:1003E4001A04019B24D4079AD2035FD4079A920378
:1003F4005ED4079A5203D2171223134018E03348ED
:10040400079A824202D11806814205D330488242BB
:1004140031D1980507402ED12A4F3A68099B9A4357
:1004240011430143396026E05200D30E069C08991B
:10043400059FBB40049A13433366099A9208F369F3
:1004440093420AD9039AD2438B6A13403E46079FCC
:10045400BA00120FB240174E26E7079F26E7032281
:10046400D20501E003229205114007229205036898
:1004740093435918016074550BB0F0BD0223D7E7BC
:100484000323D5E70523D3E70623D1E70723CFE7E3
:100494000823CDE70923CBE70A23C9E70B23C7E7E2
:1004A4000C23C5E70D23C3E70E23C1E71023BFE7E1
:1004B4001123BDE7840D0020FFFF07000400008026
:1004C40000FFFF0708270140001000B0004000B8FB
:0C04D400002000B420000020400D0300B8
:1004E000F0B5684B02225A771A68956801242543B3
:1004F00095601D6A012D43D0022D0DD0032D00D033
:100500008AE00D40042900D389E00021002D00D0AD
:1005100091E010685C77F0BD4D0813D06E1E032E7D
:1005200018D2032635400BD0468807883F04BE19F1
:100530001660012D04D0C5888688360475191560AB
:100540000D46A543C907E4D06900405A10801068E1
:100550005C77F0BD418803881B0459181160C1887D
:1005600083881B0459181160418903891B04591899
:100570001160C18983891B04591811601030E9E7A3
:100580008D0811D06D1E032D18D20E070425B60F4D
:100590000AD00678360647783F04BE1987783F02AE
:1005A000F619C778F61916600326314003295DD085
:1005B000022951D0012961D1405D5EE00178090630
:1005C00043781B04591883781B02C918C378C918CB
:1005D00011600179090643791B04591883791B02BC
:1005E000C918C379C9181160017A0906437A1B0436
:1005F0005918837A1B02C918C37AC9181160017B84
:100600000906437B1B045918837B1B02C918C37B53
:10061000C91811601030D1E700205C77F0BD016887
:1006200011604168116081681160C1681160042126
:10063000002D00D16DE7890046581660012D00D1CC
:1006400067E7401841681160022D00D161E78068BA
:10065000106010685C77F0BD41194978405D000278
:10066000401810801A6810685C77F0BD4119405D31
:1006700000024D7840191080887810701A68106850
:080680005C77F0BDBC0E002008
:10068800F0B585B0634C2178002902D0022005B06E
:10069800F0BD029203930490012626705E4A116809
:1006A80037045E4C2068C0032BD420685C4B5D1C6B
:1006B800019525601842304600D0A6E00120009040
:1006C8008604206840033CD4606800990843606051
:1006D800049802990160BFF36F8F03994160116814
:1006E800206838424DD12068019B23604C4B18424A
:1006F800009800D085E020680023304261D10020B6
:100708007FE07D20C5001068431A0320AB427CD2ED
:1007180023683B42C9D013685B1AAB4275D2236881
:100728003B42C2D013685B1AAB426ED223683B428D
:10073800BBD013685B1AAB4267D220683842E2D15B
:10074800B3E77D20C5001068431A0320AB425CD292
:1007580023683342B8D013685B1AAB4255D223687A
:100768003342B1D013685B1AAB424ED2236833428E
:10077800AAD013685B1AAB4247D220683042E2D154
:10078800A2E77D20C3001068451A03209D4238D295
:1007980025683D42A7D015686D1A9D4231D225685B
:1007A8003D42A0D015686D1A9D422AD225683D4267
:1007B80099D015686D1A9D4223D220683842E2D13B
:1007C80091E77D20C5001068471A0320AF4218D270
:1007D8002768374214D017687F1AAF4211D22768AA
:1007E80037420DD017687F1AAF420AD227683742BE
:1007F80006D017687F1AAF4203D220683042E2D190
:1008080018466168009A914361600021014A11709D
:1008180005B0F0BD8C0F00202400002010200240FD
:04082800FA8300004F
:10082C0070B52B490B6801222A480468E4030ED4E6
:10083C000468294D6E1C06602C4202D104686403C6
:10084C0025D4D10742680A434260406870BD140445
:10085C007D25ED000E68F61AAE42F2D206682642ED
:10086C00E6D00E68F61AAE42EBD206682642DFD00E
:10087C000E68F61AAE42E4D206682642D8D00E684C
:10088C00F61AAE42DDD206682642E3D1D0E79404D4
:10089C007D25ED000E68F61AAE42D2D206682642CD
:1008AC00CFD00E68F61AAE42CBD206682642C8D01C
:1008BC000E68F61AAE42C4D206682642C1D00E6843
:1008CC00F61AAE42BDD206682642E3D1B9E7C0465D
:0C08DC002400002010200240FA830000DD
:1008E80070B52B490B6801222A480468E4030ED42A
:1008F8000468294D6E1C06602C4202D1046864030A
:1009080025D4910742680A434260406870BD1404C8
:100918007D25ED000E68F61AAE42F2D20668264230
:10092800E6D00E68F61AAE42EBD206682642DFD051
:100938000E68F61AAE42E4D206682642D8D00E688F
:10094800F61AAE42DDD206682642E3D1D0E7940417
:100958007D25ED000E68F61AAE42D2D20668264210
:10096800CFD00E68F61AAE42CBD206682642C8D05F
:100978000E68F61AAE42C4D206682642C1D00E6886
:10098800F61AAE42BDD206682642E3D1B9E7C046A0
:0C0998002400002010200240FA83000020
:1009A400F0B586B06B490A78002A02D0022006B05E
:1009B400F0BD059001200870674C22680504674B60
:1009C4001968C90320D41968654E771C04971F6001
:1009D4003142014600D0B5E0012001908604186838
:1009E400400334D40022D043059908605D48007860
:1009F4005D49096808180290814200D398E000928A
:100A04007D20C200594F48E07D21CE0021688F1A15
:100A14000321B74200D395E01F682F42D3D0276843
:100A2400BF1AB74200D38DE01F682F42CBD027688E
:100A3400BF1AB74200D385E01F682F42C3D027688E
:100A4400BF1AB7427ED219682942DFD1BBE77D20A5
:100A5400C00021688F1A0321874273D21F6837426E
:100A6400C0D02768BF1A87426CD21F683742B9D0FA
:100A74002768BF1A874265D21F683742B2D02768F9
:100A8400BF1A87425ED219683142E2D1AAE70399BC
:100A9400491C02988142354F5AD058683840039116
:100AA400C9000143A81C08435860206819682942FA
:100AB4001AD021680F1A032197423CD21F682F4293
:100AC40012D027683F1A974235D21F682F420BD0A5
:100AD40027683F1A97422ED21F682F4204D02768F6
:100AE4003F1A9742E2D326E01968049F1F601C4F07
:100AF40039421FD119683142C9D021680F1A032124
:100B0400974218D21F683742C1D027683F1A9742CC
:100B140011D21F683742BAD027683F1A97420AD2C7
:100B24001F683742B3D027683F1A9742E2D302E0E6
:100B3400002103E001990598039A02605868022293
:100B4400904358600020034A1070084606B0F0BD78
:100B54000099F3E78C0F00202400002010200240AD
:100B6400FA830000900F0020600F002005E0FEFFD4
:100B7400F0B583B0814A1178002902D0022003B075
:100B8400F0BD012414700168CA077D4A0BD0416886
:100B9400012901D0202100E01C218368C5682D04AF
:100BA4001D435550016806230B40062B0BD101460B
:100BB40010312AC90D43FF208343C14359401069B2
:100BC4000840284323E08B070DD4490720D5416909
:100BD400FF239943DB434B4015691169EDB2AA2DFC
:100BE4000DD12E460CE01169664B0B40FF21C94321
:100BF400594015690D4000692843184307E0BB2696
:100C04001940CC2D00D1CC268069304308431061B3
:100C14005D4B196825041068C00326D410685B4E28
:100C2400771C029717603042204600D0A1E00120D3
:100C3400019084041068400337D40198410450683B
:100C44000091084350601968106828424DD110681B
:100C5400029D15604D4D2842019800D085E0106832
:100C64000025204261D100207FE07D20C600186865
:100C7400471A0320B7427CD217682F42CED01F6890
:100C84007F1AB74275D217682F42C7D01F687F1AE0
:100C9400B7426ED217682F42C0D01F687F1AB7427E
:100CA40067D210682842E2D1B8E77D20C7001868EF
:100CB400461A0320BE425CD216682642BDD01E6886
:100CC400761ABE4255D216682642B6D01E68761AE7
:100CD400BE424ED216682642AFD01E68761ABE4275
:100CE40047D210682042E2D1A7E77D20C7001868E8
:100CF400461A0320BE4238D216682E42A7D01E6878
:100D0400761ABE4231D216682E42A0D01E68761AD8
:100D1400BE422AD216682E4299D01E68761ABE4266
:100D240023D210682842E2D191E77D20C6001868DA
:100D3400471A0320B74218D21768274214D01F68F5
:100D44007F1AB74211D2176827420DD01F687F1A45
:100D5400B7420AD21768274206D01F687F1AB742E3
:100D640003D210682042E2D128465168009B99437F
:100D740051600021014A117003B0F0BD8C0F0020B6
:100D84001020024000604F0724000020FA83000076
:100D9400F0B58CB00F460968002900D1BCE00646C6
:100DA4005E48864201D0052000E003200090012423
:100DB40000250A950B950394029701960FE01943B9
:100DC400116039680846E040AD1C0A9A121D0A9267
:100DD4000B9A08320B92641C002800D19CE0601E20
:100DE400039B0990834019400791EAD004943E463E
:100DF40003273846A840C0432C4675682946394025
:100E04004A1E012A0695059413D808900198826811
:100E1400089F3A40F7680646A74017438760EA06EA
:100E2400D20F09988240089877689F4317437760E8
:100E340007E00329019E04D1029F2B462546049C0A
:100E44001FE0F2680240029FBB682546A34013439B
:100E5400F3600229069B049C13D108901C200A9974
:100E640008400F218140099AD2089200B218136AEF
:100E74008B43396981400898194311627B680321C7
:100E84001940A940326802400A4332609803800F37
:100E940097D0032009998143214840180521090767
:100EA4008E42016E0AD0204A964205D01F4A9642CD
:100EB400009B04D1022302E0012300E00023182256
:100EC4000B9E32400F269640B143603093400B4353
:100ED4000360134801687868C20202D5079B19436E
:100EE40001E0079B99430E4A11605168820201D5C3
:100EF400194300E099430A4A51600A494968820348
:100F040001D5194300E09943064A51601168C003B2
:100F140000D554E7994353E70CB0F0BD000C0050E2
:100F240000180240801802400004005000080050DD
:100F3400F0B585B003AD00242C70384F3E689B1B80
:100F44009E18374A1268232353431A0D72433D46B1
:100F54003F680492029003689A680A421AD00322F6
:100F640001925202914218D10094284602E09968F5
:100F740011424DD0197B03AC217003990168C91B40
:100F8400B1421DD20499049C641E04940029EED13C
:100F94000026ECE7002005B0F0BD284603E09A687F
:100FA4000A422C4637D00268D21BB24208D22546E8
:100FB400049A049C641E0494002AF0D10026EEE7EF
:100FC4005968E0229143596041218900029842689E
:100FD4008A420BD181680122D403A14202D0920239
:100FE400914203D1196840229143196001214A03B7
:100FF400846A5C30944205D11C6894431C601C686C
:1010040014431C60002202704170019805B0F0BDC9
:10101400009805B0F0BD204605B0F0BD24000020C6
:041024002000002088
:10102800F0B582B0254C2368D21A551824490968AE
:101038004901090D694326680191026893680021F6
:101048001B0637D503465C33009302E093681B0602
:1010580030D52768BF1BAF4207D2019F019B5B1E9B
:101068000193002FF2D10025F0E75168E024A14355
:1010780051604121890044688C420BD18168012468
:10108800E503A94202D0A402A14203D11168402479
:10109800A143116001214C03806AA04205D1106868
:1010A800A04310601068204310600020009A107060
:1010B80051700321084602B0F0BDC046240000204C
:0410C80020000020E4
:1010CC00F0B589B05C249C4E335D012B00D131E12D
:1010DC00012705943755994B1B6806935D230493A0
:1010EC00F35C012B6FD1002800D120E1002900D145
:1010FC001DE1049BF35C042B02D00523049C3355A7
:10110C000390002333664625725344243253F287EE
:10111C00F4688B48029484423C4600D30024240398
:10112C000194380337687C6884430020019BE418E1
:10113C007C603164039BB363F0643065B2873A68BA
:10114C00520603D43A68402313433B60029A7C4B0B
:10115C009A427268069C43D3002A039806D10288EF
:10116C00FA60801CB063F28F521EF287012205E0F8
:10117C00724B1B681B1B0A2B00D3D5E0F38F002B83
:10118C0002D1735B002B6AD0BB689B070CD5F38F25
:10119C00002B09D0012A07D10288FA60801CB063A9
:1011AC00F28F521EF2870022BB68DB07E0D0735B24
:1011BC00002BDDD0FA680A80725B521E7253891CB8
:1011CC0031640122D4E74124A4007568A54200D003
:1011DC00ADE0042B00D0AAE0B368002B83D0A6E0CE
:1011EC00002A039807D100783873B06B401CB063A9
:1011FC00F08F401EF087012005E050490968091B5B
:10120C000A2900D390E0F18F002901D0376803E060
:10121C00715B0029376822D0B96889070ED5F18F28
:10122C0000290BD0012809D1B06B00783873B06B52
:10123C00401CB063F08F401EF0870020B968C907CE
:10124C00DBD0715B0029D8D0387B316C0870705BB7
:10125C00401E7053306C401C30640120CDE707A851
:10126C000021039101703748006823214143090D87
:10127C00324A1068201A0A3041431268089103253B
:10128C00B968C904890F12D0EB0203E0B96819429E
:10129C00069C0CD029490968891A814217D20899F1
:1012AC00089C641E08940029F0D10020EEE7224827
:1012BC000A212246FFF7B2FE00282DD169021E48F2
:1012CC000A222346FFF730FE002825D129E0786852
:1012DC00E0218843786041208000716881420BD105
:1012EC00B1680120C203914202D08002814203D135
:1012FC00386840218843386001214A03B06A904223
:10130C00059B05D1386890433860386810433860C5
:10131C000398F05404983154306E20210843306601
:10132C003166306E002802D10120049970540020DF
:10133C000599705409B0F0BD200D00202400002048
:08134C00010700002000002051
:1013540070B58021415821291AD102465632938A08
:10136400002B15D00168104C02E05B1E1D040FD049
:101374001588002D0DD0CD692D06F6D5056D2E8866
:1013840026408E62AD1C056515886D1E1580ECE740
:1013940070BD0120C0058A6882438A6008684022C3
:0C13A40002430A6070BDC046FF0100005B
:1013B00030B58023C15821290FD1024656321188F9
:1013C000002901680AD0036D1C88084D25408D62F4
:1013D000991C01651088401E108030BD0868984334
:1013E00008600868402202430A6030BDFF01000027
:1013F000F0B584B084214158222920D101465E31C4
:101400004E89320400D184E00246843203924B8834
:1014100003253540846D16D007687F6A1F4027700A
:101420000C88641E0C80846D641C84650F88002FFA
:101430000DD0012D23D1751E042E6AD380E00068E3
:101440001830082174E03546042E79D261E0012776
:101450003A020292026800921768029A9743009A31
:1014600017600196966802966C4F3740019E976010
:101470000027C7662027039A1760012DDBD0076875
:101480007F6A1F4027700C88641E0C80846D641C6A
:1014900084650F88002F05D0022D1BD1B51E042EA8
:1014A0004ED236E001273A02029202680092176893
:1014B000029A9743009A1760019595680295574FD5
:1014C0002F40019D97600027C7662027039A176069
:1014D000022DE3D005686D6A1D4025700C88641EDE
:1014E0000C80846D641C84650D88002D0ED101254F
:1014F0002A0207683D6895433D60BA68474D15402C
:10150000BD600025C5662025039A1560F51E042ED2
:1015100016D20A88002A0ED049898A420BD2414944
:10152000C1663E49491C006882680A4082602021E9
:1015300002680A43026004B0F0BD2D1F2E04E8D0FB
:101540000668766A1E4026700C88641E0C80846DC6
:10155000641C84650E88002E0DD106683768304AF9
:1015600017403760B7682D4A1740B7600026C66637
:101570002026039A16600668766A1E4026700C883C
:10158000641E0C80846D641C84650E88002E0DD151
:1015900006683768224A17403760B7681F4A174005
:1015A000B7600026C6662026039A16600668766A2B
:1015B0001E4026700C88641E0C80846D641C84653B
:1015C0000E88002E0DD106683768154A174037601F
:1015D000B768124A1740B7600026C6662026039AED
:1015E00016600668766A1E4026700C88641E0C80A1
:1015F000846D641C84650E88002E9ED10668376851
:10160000074A17403760B768044A1740B76000269A
:10161000C6662026039A16608FE7C046FEFFFFEFDE
:08162000FFFEFFFF51BD0008B1
:10162800F0B583B084214158222922D101465E3188
:101638004F893A0477D00246843202924B880326B7
:101648003E40856D046818D00197676A1F402F8057
:101658000F887F1E0F80AA1C009282650F88002FBA
:101668000FD0012E1DD1019F7E1E009D042F71D227
:1016780059E000681830082164E03E46042F69D21A
:1016880051E001273A02276897432760A268624F12
:101698001740A7600027C7662027029A1760012E07
:1016A800E1D0676A1F406F800F887F1E0F802A1D58
:1016B800009282650F88002F07D0022E019F15D156
:1016C800BE1E009D042F45D22DE001273A0227684F
:1016D80097432760A268504F1740A7600027C76646
:1016E8002027029A1760022E019FE9D0666A1E40E1
:1016F800AE800E88761E0E80AD1D85650E88002E84
:101708000ED1012636022768B7432760A668424FE4
:101718003740A760019F0026C6662026029A1660F9
:10172800FE1E042F16D20A88002A0ED049898A4242
:101738000BD23B49C1663849491C006882680A4097
:101748008260202102680A43026003B0F0BD361FA0
:101758003704E8D0676A1F402F800F887F1E0F80EC
:10176800AD1C85650F88002F0CD127682B4A1740C0
:101778002760A768284A1740A7600027C766202760
:10178800029A1760676A1F402F800F887F1E0F809C
:10179800AD1C85650F88002F0CD127681F4A17409C
:1017A8002760A7681C4A1740A7600027C76620273C
:1017B800029A1760676A1F402F800F887F1E0F806C
:1017C800AD1C85650F88002F0CD12768134A174078
:1017D8002760A768104A1740A7600027C766202718
:1017E800029A1760676A1F402F800F887F1E0F803C
:1017F800AD1C85650F88002FA9D12768074A1740B7
:101808002760A768044A1740A7600027C7662027F3
:10181800029A17609BE7C046FEFFFFEFFFFEFFFF3F
:0418280097C100085C
:10182C00F0B586B0012041044A4A13680B4313609B
:10183C0012680A40059205993D25474B02210491F7
:10184C005955464A1646183E1E609168444C214232
:10185C0006D19168434C214202D1316881433160F9
:10186C004821002402915C543E2101915C541F4696
:10187C003E377C70BC70FC703C717C7144210091D3
:10188C005C54194644314C708C70CC705C55364AA3
:10189C005C609C60DA601C611A462B46555D002D1D
:1018AC0001D13C2554551546049A0393EA542B4612
:1018BC000725ED013268AA439D6915433560274D14
:1018CC00294A6A612C615A69AA612A1F10602E4646
:1018DC00083E3268D20702D0326882433260029AE4
:1018EC009854019A98547870B870F870387178716F
:1018FC00009A985448708870C87003995854A96815
:10190C00AA688243AA602A6802432E46F025AA439D
:10191C0032600A229143B16031680C2291433160EC
:10192C00316811433160316D049A11430D2291439A
:10193C0031653C215C54FF2109020C4A13688B432E
:10194C00136040050A490860BFF34F8FBFF36F8FD8
:10195C0006B0F0BD40100240440E00201844014077
:10196C001111000044040000FFFF000014E400E02B
:04197C0080E100E026
:10198000F0B581B0017F012953D12B4C2168012989
:1019900005D10068406B2E490860022048E02168AC
:1019A000022946D101684A6B24490A600122530585
:1019B000234D2B60BFF34F8FBFF36F8F214B1E68FA
:1019C000F7680225AF43F760376A97433762376A93
:1019D0003762376A1C490F4206D1316A1B4F3942C0
:1019E00002D13168914331603E215A5444215A5406
:1019F000E94300680161164800681049096881429E
:101A000001D9081A03E0FED2081A124940181249F7
:101A10000860086800031149884208D2104807F09E
:101A200083FF0D48006801030E4809F0A7F8032062
:101A3000206001B0F0BDC0466C0F0020500F0020A8
:101A400080E100E0440E0020111100004404000079
:101A5000540F0020FFFF0000700F0020405DC60003
:081A6000A4C9000802C7000838
:101A6800F0B58DB00120089005037B4F3D607B4C9D
:101A780020682168091A96290BD82168091A96291D
:101A880007D82168091A962903D82168091A9729BD
:101A9800EFD3734820210161226823689B1A962B93
:101AA8000BD823689B1A962B07D823689B1A962B6A
:101AB80003D823689B1A972BEFD30160206821680D
:101AC800091A96290BD82168091A962907D8216876
:101AD800091A962903D82168091A9729EFD33D6175
:101AE800FF2000065F490A688243089BD807101840
:101AF80008605D488021016005950BAD00200690C7
:101B0800A8705A482880DE033E61022228462946EA
:101B1800FFF7D8FA3E60262028703E610322284647
:101B28002946FFF7CFFA07963E60A8780A283DD1E4
:101B380020682168091A96290BD82168091A96295C
:101B480007D82168091A962903D82168091A9729FC
:101B5800EFD3079E3E610BAD22272F70032204921C
:101B680028462946FFF7AEFA3B480660422028700F
:101B780039480661A878072101402031697002229E
:101B880028462946FFF79EFA334806602F70074615
:101B98003E6128462946049AFFF794FA3E60A878E1
:101BA800800607D4324807F0BBFEFEE7314807F04D
:101BB800B7FEFEE735463E610BAF23203870064678
:101BC80004900322039238463946FFF77BFA2249EC
:101BD8000D604320019038700D61B878EF21014005
:101BE80079700222029238463946FFF76BFA1A4892
:101BF80005603E70056138463946039E3246FFF758
:101C080061FA1548056005610BAF049838703846CD
:101C180039463246FFF756FA0F4E3560019838704C
:101C28003561B8789F2101402031797038463946AE
:101C3800029AFFF747FA35600498387035613846DC
:101C48003946039AFFF73EFA3560B878800615D40E
:101C5800094807F065FEFEE7180000502400002040
:101C68001804005004E400E000E100E0460A000027
:101C7800B8C30008E4C90008D3C300080BAD069830
:101C8800A8703420687051202870079F376102229D
:101C980028462946FFF716FA376031202870376141
:101CA800032228462946FFF70DFA3760A87834281A
:101CB80002D0F84807F034FE0BA8069A8270F6495D
:101CC800018009ADAA702A80376103222946FFF7EF
:101CD800F9F937602878FF2805D10BA8007809A9F9
:101CE800497881425DD00BA8069A8270EA49018042
:101CF80009ADAA702A80376103222946FFF7E2F965
:101D080037602878FF2805D10BA8007809A94978F9
:101D1800814246D00BA8069A8270DF49018009AD3E
:101D2800AA702A80376103222946FFF7CBF937606A
:101D38002878FF2805D10BA8007809A9497881429D
:101D48002FD00BA8069A8270D349018009ADAA70DA
:101D58002A80376103222946FFF7B4F937602878CB
:101D6800FF2805D10BA8007809A94978814218D025
:101D78000BA8069A8270C849018009ADAA702A800A
:101D8800376103222946FFF79DF937602878FF2835
:101D980000D09DE00BA8007809A94978814200D0BD
:101DA80096E009A885786020029005430BA8457045
:101DB800452103910170376109AE069931800222ED
:101DC80031460492FFF77EF9B44807603078FF285F
:101DD80005D10BA8007809A9497881425ED00BA8E3
:101DE800457003990170AD490F6109AE06993180BC
:101DF80002223146FFF766F9A84807603078FF28C5
:101E080005D10BA8007809A94978814246D00BA8CA
:101E1800457003990170A1490F6109AE0699318097
:101E280002223146FFF74EF99C4807603078FF28B8
:101E380005D10BA8007809A9497881422ED00BA8B2
:101E480045700399017095490F6109AE0699318073
:101E580002223146FFF736F9904807603078FF28AC
:101E680005D10BA8007809A94978814216D00BA89A
:101E7800457003990170894D2F6109AE069931802B
:101E880002223146FFF71EF92F603078FF283CD137
:101E98000BA8007809A94978814236D1804D049869
:101EA80068770BA8069B838028688168089A114385
:101EB800816079490B912A6A09A9012A45D0022A29
:101EC80040D0032A1A4643D1734A02600C9A3AE07A
:101ED8000899C802C906321F1268130402400B4051
:101EE8009A1842403260226823689B1AC82BF2D89D
:101EF80023689B1AC82BEED823689B1AC82BEAD8EC
:101F080023689B1AC82BEFD9E5E70899C802C906C8
:101F18002A1F1268130402400B409A1842402A6094
:101F2800226823689B1AFA2BF2D823689B1AFA2B8B
:101F3800EED823689B1AFA2BEAD823689B1AFA2B47
:101F4800EFD9E5E7574A026001E0574A0280026884
:101F5800081D03900BA882700899697709AFBB80A8
:101F680009934E4D079E2E6106223946FFF7AAF8BF
:101F78002E603878FF2820D10BA8007809A9497865
:101F880081421AD10BA8407809A98978814214D1D5
:101F98000BA8807809A9C97881420ED109A845798A
:101FA80001210398FEF798FAA84206D109A80079FA
:101FB80002990840602800D160E10498384D68779C
:101FC8000BA80021818028688268089B1A438260D8
:101FD800314A0B922A6A012A0BD0022A06D0032A18
:101FE8000A4609D12C4A02600C9A00E02D4A026088
:101FF80001E02D4A028002680BA882706B7709AF56
:10200800B9800991254D2E6106223946FFF75AF805
:102018002E603878FF2820D10BA8007809A94978C4
:1020280081421AD10BA8407809A98978814214D134
:102038000BA8807809A9C97881420ED109A84579E9
:1020480001210398FEF748FAA84206D109A80079A9
:1020580002990840602800D110E10498104D687773
:102068000BA80021818028688268089B1A43826037
:10207800094A0B922A6A012A18D0022A06D0032A92
:102088000A4616D1044A02600C9A00E0054A02602A
:102098000EE0C046ECC5000825EC00001800005012
:1020A800BC0E0020000025ECEC2500004F4A028001
:1020B80002680BA882706B7709AFB98009914C4D03
:1020C8002E6106223946FEF7FDFF2E603878FF287C
:1020D80020D10BA8007809A9497881421AD10BA808
:1020E800407809A98978814214D10BA8807809A978
:1020F800C97881420ED109A8457901210398FEF7D4
:10210800EBF9A84206D109A800790299084060288D
:1021180000D1B3E00498374D68770BA8002181807F
:1021280028688268089B1A438260334A0B922A6A9D
:10213800012A0BD0022A06D0032A0A4609D12E4AC0
:1021480002600C9A00E02D4A026001E0274A0280F2
:1021580002680BA882706B7709AFB9800991244D8A
:102168002E6106223946FEF7ADFF2E603878FF282B
:102178001FD10BA8007809A94978814219D10BA869
:10218800407809A98978814213D10BA8807809A9D8
:10219800C97881420DD109A8457901210398FEF734
:1021A8009BF9A84205D109A800790299084060283E
:1021B80064D004980F4D68770BA8002181802868A7
:1021C8008268089B1A4382600B4A0B922A6A012A8A
:1021D80016D0022A064F06D0032A0A4619D1064A03
:1021E80002600C9A00E0054A026011E0EC2500004C
:1021F80018000050BC0E002025EC0000000025EC63
:10220800014A0280014F03E0EC250000180000504D
:1022180002680BA882706B7709ADA98009913E61AD
:1022280006222946FEF74EFF3E602878FF2800D098
:1022380062E20BA8007809A94978814200D05BE2E4
:102248000BA8407809A98978814200D054E20BA8EC
:10225800807809A9C978814200D04DE209A845795A
:1022680001210398FEF738F9A84200D044E209A8F2
:10227800007902990840602800D03DE20E48CD3030
:1022880004900B900BAE02213046FEF725F9B07092
:102298000020069009900948079D056109AF0422AE
:1022A800304639460392FEF70DFF0448056038783A
:1022B800FF2818D104E0C04625EC000018000050A3
:1022C8000BA8007809A9497881420CD10BA840785D
:1022D80009A98978814206D10BA8807809A9C9780B
:1022E800814200D1A7E004980B900BAE0221304642
:1022F800FEF7F2F8B07006980990FE48056109AF3C
:10230800042230463946FEF7DDFEFA480560387883
:10231800FF2811D10BA8007809A9497881420BD16F
:102328000BA8407809A98978814205D10BA8807843
:1023380009A9C97881427ED004980B900BAE02217E
:102348003046FEF7C9F8B07006980990E94805616B
:1023580009AF042230463946FEF7B4FEE548056069
:102368003878FF2811D10BA8007809A9497881424B
:102378000BD10BA8407809A98978814205D10BA80F
:10238800807809A9C978814255D004980B900BAE82
:1023980002213046FEF7A0F8B07006980990D5489B
:1023A800056109AF042230463946FEF78BFEFE4828
:1023B80005603878FF2811D10BA8007809A9497859
:1023C80081420BD10BA8407809A98978814205D1AF
:1023D8000BA8807809A9C97881422CD004980B9061
:1023E8000BAE02213046FEF777F8B07006980990D8
:1023F800ED48056109AF042230463946FEF762FE12
:10240800E94805603878FF2800D095E10BA80078E6
:1024180009A94978814200D08EE10BA8407809A922
:102428008978814200D087E10BA8807809A9C9780A
:10243800814200D080E10BAE069DB580DB480B9051
:1024480002213046FEF748F8B07009AFBD80099503
:10245800D548079D0561062230463946FEF732FE0B
:10246800D1480560381D04903878FF2824D10BA87E
:10247800007809A9497881421ED10BA8407809A99A
:102488008978814218D10BA8807809A9C978814236
:1024980012D109AE7579012704983946FEF71CF860
:1024A800401B411E884103997156002900DA002714
:1024B8003843012800D061E10BAF069DBD80BB48C1
:1024C8000B9002213846FEF707F8B87009AEB580C0
:1024D8000995B548079D0561062238463146FEF73D
:1024E800F1FDB14805603078FF2824D10BA80078A9
:1024F80009A9497881421ED10BA8407809A9897891
:10250800814218D10BA8807809A9C978814212D1D3
:1025180009AE7579012704983946FDF7DDFF401BA0
:10252800411E884103997156002900DA0027384373
:10253800012800D022E10BAF069DBD809B480B907F
:1025480002213846FDF7C8FFB87009AEB580099575
:102558009548079D0561062238463146FEF7B2FDCB
:10256800914805603078FF2824D10BA8007809A984
:10257800497881421ED10BA8407809A989788142FF
:1025880018D10BA8807809A9C978814212D109AE5F
:102598007579012704983946FDF79EFF401B411EB7
:1025A800884103997156002900DA00273843012829
:1025B80000D0E3E00BAF069DBD807C480B90022164
:1025C8003846FDF789FFB87009AEB5800995764899
:1025D800079D0561062238463146FEF773FD7248AD
:1025E80005603078FF2824D10BA8007809A949781C
:1025F80081421ED10BA8407809A98978814218D157
:102608000BA8807809A9C978814212D109AE7579D9
:10261800012704983946FDF75FFF401B411E88419A
:1026280003997156002900DA00273843012800D0A1
:10263800A4E00BAF069DBD805C480B900221384694
:10264800FDF74AFFB87009AEB58009955648079D51
:102658000561062238463146FEF734FD52480560CA
:102668003078FF2823D10BA8007809A9497881423E
:102678001DD10BA8407809A98978814217D10BA8E8
:10268800807809A9C978814211D109AE777904986F
:10269800089D2946FDF720FFC01B411E884103996C
:1026A8007156002900DA069D2843012866D14B207F
:1026B8008000089AD102D2063B4F3B1F1B681D04BD
:1026C8000B401540EB184B403B6023682568EE1A19
:1026D80005466435AE42F0D82668F61AAE42ECD804
:1026E8002668F61AAE42E8D82668F61AAE42EDD940
:1026F800E3E7C046180000504B208000089AD1023A
:10270800D2063E46331F1B681D040B401540EB18CC
:102718004B40336023682568ED1A8542F2D8256856
:10272800ED1A8542EED82568ED1A8542EAD8256863
:10273800ED1A8542EFD9E5E74B208000089AD102CF
:10274800D206194F3B1F1B681D040B401540EB18A0
:102758004B403B6023682568EE1A05463235AE4289
:10276800F0D82668F61AAE42ECD82668F61AAE42B9
:10277800E8D82668F61AAE42EDD9E3E72068216862
:10278800091A96290BD82168091A962907D82168A9
:10279800091A962903D82168091A9729EFD30248FC
:1027A800059901600DB0F0BD1800005021EC000043
:1027B800F0B583B0B44807F0B3F8B44D01262E84C1
:1027C80037044B200002A861EF6128462A301E21F9
:1027D80009F07AF9B820AE492950F920C0433230BF
:1027E800B6216852B42032212952B020A949295073
:1027F800AC20A94A2A50A8202950A4202A50A02059
:10280800A64929509C20A64929509820A549295015
:1028180096210220685294216E549021A24A6A504F
:102828008821A24A6A508021A14A6A502946183153
:10283800A04A4A67A04ACA66A04A0021A04BAB64D6
:10284800E96429656965AA65BC22A950D022A95006
:10285800CC225A23AB522A46BC3251609160D160D7
:10286800CA43984BC043984C29666966AA66EA66CB
:102878002C676A67AB67E867D820686039202870DA
:10288800A868401CA860914C6068002806D52046BE
:1028980008388F4901608F49016060688E48006878
:1028A8002168C9031FD421688C4A531C2360114234
:1028B80002D1216849036FD46068C00702D06068FC
:1028C800B043606086480670864C206886490E7062
:1028D8000006400E401E8549086002A8FEF75EF813
:1028E800002823D0FEE77D21C9007B4A1268121A0E
:1028F8008A42E1D222683A42D5D0774A1268121A3F
:102908008A42D9D222683A42CDD0734A1268121A42
:102918008A42D1D222683A42C5D06F4A1268121A46
:102928008A42C9D222683A42DFD1BCE700970196B1
:1029380020680006800B6E4E8419FF2087020CCD9C
:102948002046083DFDF79CFE0028FED1654800683A
:10295800800238403018D430083508348442EED329
:102968005D48006859490968009B1942019C3CD19F
:10297800564D2968594A531C2B60114202D12968C7
:10298800490359D4E007514A5168014351605068DE
:1029980000F0B0F803B0F0BDB1047D22D2004E4B78
:1029A8001B681B1A934287D223680B4284D04A4B78
:1029B8001B681B1A934200D37EE723680B4200D1A1
:1029C8007AE7454B1B681B1A934200D374E72368C8
:1029D8000B4200D170E7404B1B681B1A934200D38F
:1029E8006AE723680B42DAD166E77D21C9003A4AD3
:1029F8001268121A8A42C5D2344A12681A42B7D0EB
:102A0800354A1268121A8A42BCD2304A12681A42EF
:102A1800AED0314A1268121A8A42B3D22B4A1268CF
:102A28001A42A5D02C4A1268121A8A42AAD2274AF8
:102A380012681A42DBD19BE7A1047D22D200264B03
:102A48001B681B1A93429DD2204B1B680B4299D0DE
:102A5800214B1B681B1A934294D21C4B1B680B42D8
:102A680090D01D4B1B681B1A93428BD2174B1B68C7
:102A78000B4287D0184B1B681B1A934282D2134B08
:102A88001B680B42DBD17DE7BEC70008E0030020CE
:102A98001027070054F248F44C1D581B06FFFA0093
:102AA800983AB036E02ED430B036D430804828007A
:102AB800630069000A000200A086010040420F007E
:102AC80090D00300007884C900D68AEA102002401A
:102AD80023016745AB89EFCD24000020FA8300006D
:102AE800940F0020E075FF1F900F0020600F00205A
:042AF80000F8FF07DC
:102AFC00F0B598B0DC4800680006800BDB49411843
:102B0C00481C1790881C1690C81C1590081D149012
:102B1C00481D1390881D1290C81D1190084608304E
:102B2C001090084609300F9008460A300E9008465F
:102B3C000B300D9008460C300C9008460D300B9065
:102B4C0008460E300A9008460F300990084610309F
:102B5C000890084611300790084612300690084637
:102B6C001330059008461430049008461530039035
:102B7C000846163002900846173001900846183067
:102B8C0000900D4619350E461A36D720C743B84863
:102B9C00C019CB19D8229B5C8354179BDB199B5C07
:102BAC00D9240355169BDB199B5CDA240355159B22
:102BBC00DB199B5CDB240355149BDB199B5CDC242D
:102BCC000355139BDB199B5CDD240355129BDB190E
:102BDC009B5CDE240355119BDB199B5CDF240355A6
:102BEC00109BDB199B5CE02403550F9BDB199B5C52
:102BFC00E12403550E9BDB199B5CE22403550D9BD2
:102C0C00DB199B5CE32403550C9BDB199B5CE424D4
:102C1C0003550B9BDB199B5CE52403550A9BDB19C5
:102C2C009B5CE6240355099BDB199B5CE72403554D
:102C3C00089BDB199B5CE8240355079BDB199B5C09
:102C4C00E9240355069BDB199B5CEA240355059B81
:102C5C00DB199B5CEB240355049BDB199B5CEC247C
:102C6C000355039BDB199B5CED240355029BDB197D
:102C7C009B5CEE240355019BDB199B5CEF240355F5
:102C8C00009BDB199B5CF0240355EB199B5CF12436
:102C9C000355F3199A5CF223C2541B3700D076E724
:102CAC0073498869734C2061888BA082C88BE08241
:102CBC00088C2083488CA083888CE083C88C20846B
:102CCC00088D6084488D7C22A052888D7E22A05273
:102CDC00C88D98221692A052088E9A221492A05255
:102CEC00488E8C221292A052888EA0221592A0524D
:102CFC00C88EA8221792A0520A463832ECCAC86C69
:102D0C001390086D1090486D0F90802022508422F3
:102D1C00A3508822A55090231193E6509C26A751CE
:102D2C00A425139B6351AC231393109FE7500F9B67
:102D3C00A3678F6D9423E750085A5227E0538220E3
:102D4C00085A5027E05308461830C06EE065885882
:102D5C0020661298085A5422A0528E20085A5622E5
:102D6C00A0521198085A5822A0529220085A5A225E
:102D7C00A052C85C6422A0529620085A6822A05225
:102D8C001698085AA0861498085AE086885B208703
:102D9C009E20085A60871598085AA087A220085AC6
:102DAC00E087485B4022A052A620085A4222A0523B
:102DBC001798085A4422A052AA20085A4622A05218
:102DCC001398085A4822A052AE20085A4A22A05200
:102DDC00B020085A4C22A052B220085A4E22A052BF
:102DEC00B420085A6A22A052B620085A6C22A0526B
:102DFC00B820085A6E22A052BA20085A7022A0524B
:102E0C00BC200A582046C8304266C0228A588266C6
:102E1C00C4228A58C266C8228A580267CC228A5AAF
:102E2C007223E252D0228A5802660A6E15924B6EB9
:102E3C000A46683264CA14964F6F8E6F1696CE6F20
:102E4C0017964363159B036342648564C767149AA2
:102E5C0082672920C000169A225020184660C86844
:102E6C00606018B0F0BDC046E075FF1F00F8FF07AA
:082E7C00E00300202800002003
:102E8400F0B59DB00390E24806F04CFDE1480068BF
:102E94000006800BE0494218501C1B90901C1A90AD
:102EA400D01C1990101D1890501D1790901D16904D
:102EB400D01D159010460830149010460930139018
:102EC40010460A30129010460B30119010460C3008
:102ED400109010460D300F9010460E300E90104694
:102EE4000F300D90104610300C90104611300B909E
:102EF400104612300A9010461330099010461430D0
:102F0400089010461530079010461630069010466B
:102F14001730059010461830049011461931FF23DC
:102F24009B02029300230193DC430094CF3CBB4BF0
:102F34001D191619D023F65CEE541B980619F65C7D
:102F4400D127EE551A980619F65CD227EE55199832
:102F54000619F65CD327EE5518980619F65CD427A3
:102F6400EE5517980619F65CD527EE5516980619EE
:102F7400F65CD627EE5515980619F65CD727EE555C
:102F840014980619F65CD8202E54139E3619F65C54
:102F9400D927EE55129E3619F65CDA27EE55119EA6
:102FA4003619F65CDB27EE55109E3619F65CDC27E5
:102FB400EE550F9E3619F65CDD27EE550E9E36193A
:102FC400F65CDE27EE550D9E3619F65CDF27EE55CE
:102FD4000C9E3619F65CE027EE550B9E3619F65C0E
:102FE400E127EE550A9E3619F65CE227EE55099E56
:102FF4003619F65CE327EE55089E3619F65CE4278D
:10300400EE55079E3619F65CE527EE55069E3619F1
:10301400F65CE627EE55059E3619F65CE727EE5575
:10302400049E3619F65CE827EE550E19F65CE9277E
:10303400EE557A4D1A3400D079E71A90686D784EBF
:103044007065688D7085A88DB085686B1990294668
:10305400383116C9686C1B90AF6CE86C1890286DF9
:103064001790688E7086A86DB065E88DF085288EFF
:10307400308619987063B163F26334641B9870648A
:10308400B7641898F06417983065039F012F01D036
:10309400A86901E04B2000020199B061012F0846A4
:1030A40000D0A88BB083012F03D1F78304D1632010
:1030B40004E0E88BF083FAD07820285A2A8C802107
:1030C4007052012F06D0685888217050012F05D105
:1030D4000A2405E0534888217050F9E784202C5ACB
:1030E4008C2019903452012F06D07A242C5B82252F
:1030F4007453012F03D003E06924822574533A46A4
:103104003284012F01980246444D0CD17284024648
:103114000DD1B284012F02460ED1F28402463285CB
:1031240013E0EA6F12E06A8C72840246F1D0AA8C32
:10313400B284012F0246F0D0EA8CF284012F0246B9
:10314400EDD02A8D3285012FEBD1374A344618341D
:10315400E2660222012F1B9201D08622AA5A8E20F7
:1031640018903252314C012F00D06C5A9022B45234
:103174002F49012F0C4601D08A242C5B92201790F2
:1031840034523846012F01D1054601E0199C2D5DCA
:103194009424355501281B98FD4D01D01898285AC0
:1031A40096271997F0530398012805D0AA5A982511
:1031B4007253012804D106E0F74A9825725302E0BD
:1031C400F3481799415A9A27F1530398012802D0DA
:1031D400EF48025B00E0F14AEE4C9C2172520398E6
:1031E400012802D0EA48199A845A9E203452F922BE
:1031F400D443039A012A1994224601D0E44A525B2B
:10320400A0243253039A012A14D0E14AD25B12E07B
:1032140035C40008E075FF1F00F8FF07B80400205C
:10322400E003002080482800A0860100B03600009A
:10323400D4300000FA22A22417943253D84A039DB2
:10324400012D01D0D24A525AA42116917252D0496A
:103254000A5AD449012D084600D01046A8271897C9
:10326400F053D148012D054600D01546A622B5528B
:10327400CE4F039D012D3D4601D0C54D2D5BAA24A3
:1032840017943553039D012DC54C02D0C04C169D97
:10329400645BAC257453039C012C01D0BC48805A58
:1032A400AE2430530398012802D0B9481899415AE2
:1032B400B02031520399012902D0B549179A8F5A87
:1032C400B222B752039F012F02D0B1494D5B00E0F7
:1032D4003225B42118917552012F02D0AC4D295BCF
:1032E40001E019993231019DB6243153012F07D0E1
:1032F400A74C245AB8203452012F05D1072205E0E7
:10330400AB4CB8203452F9E7A14CA25ABA24325338
:10331400012F2A4602D09E4A18995258BC21725055
:10332400012F2946984C01D099490958C0203150A1
:10333400C420012F02D09649095A00E05A21CC2218
:10334400B152C821012F2A4601D0914A5258F25055
:10335400755035501B98C0439649974A3566756633
:10336400009BB366F36632677367B167F067884999
:103374008868401C88601A997160B0603920307088
:10338400012F284601D08248007C3074012F01D0DF
:103394007F48C568F560894D6868002806D52846C9
:1033A4000838874901608749016068688648006871
:1033B40001211B910F042968C9031FD42968834A7A
:1033C400531C2B60114202D1296849036AD46868EE
:1033D400C0071B9A02D06868904368607C480270FA
:1033E40020687C490A700006400E401E7A49086035
:1033F4001CA8FDF7D5FA002823D0FEE77D21C900DB
:10340400714A1268121A8A42E1D22A683A42D5D025
:103414006D4A1268121A8A42D9D22A683A42CDD029
:10342400694A1268121A8A42D1D22A683A42C5D02D
:10343400654A1268121A8A42C9D22A683A42DFD10E
:10344400BCE72068800202990840504944180CCE19
:103454002046083EFDF716F90028FED14A480068C8
:1034640080020299084049490818D43008360834C3
:103474008442ECD354480068296839423BD1296816
:10348400524A531C2B60114202D12968490355D476
:103494001B98C0076968014369606868FFF72CFBE3
:1034A4001DB0F0BD1B9989047D22D200464B1B68D8
:1034B4001B1A93428BD22B680B4288D0424B1B6859
:1034C4001B1A934283D22B680B4200D17FE73E4BF9
:1034D4001B681B1A934200D379E72B680B4200D177
:1034E40075E7394B1B681B1A934200D36FE72B68AF
:1034F4000B42DBD16BE77D21C900334A1268121AF3
:103504008A42C5D22A683A42B9D02F4A1268121A9E
:103514008A42BDD22A683A42B1D02B4A1268121AA2
:103524008A42B5D22A683A42A9D0274A1268121AA6
:103534008A42ADD22A683A42DFD1A0E71B998904B6
:103544007D22D200204B1B681B1A9342A0D22B6809
:103554000B429DD01C4B1B681B1A934298D22B68BC
:103564000B4295D0184B1B681B1A934290D22B68C0
:103574000B428DD0144B1B681B1A934288D22B68C4
:103584000B42DFD184E7C046E075FF1F00F8FF0758
:10359400B8040020B0360000E02E0000983A000085
:1035A4004C1D000054F2FFFF581B000048F4FFFFBD
:1035B40010270000007884C900D68AEA102002404F
:1035C40023016745AB89EFCD24000020FA83000076
:0C35D400940F0020900F0020600F0020DA
:1035E000F0B591B00F90F14806F09EF9F04E3069B9
:1035F000F04DA861B08AA883F08AE883308B2884D4
:10360000B08B6884F08BA884308CE884708C28851B
:103610007E20305AA8857C20305A688598200C90EE
:10362000305AE8859A200A90305A28868C200790D4
:10363000305A6886A0200B90305AA886A8200E9099
:10364000305AE8868024305904908422B058039080
:1036500088200590305802909020069030580190B4
:103660009C2008903358A42009903258AC200D902B
:103670003058B16F049FAF63039FEF63029F2F64C5
:10368000019F6F64AB64EA642865696594203158D2
:10369000A9655221715A29535021715A8222A95287
:1036A000F16D2A461832D166316E059AA95054211F
:1036B000715A079AA9525621715A8E22A95258213D
:1036C000715A069AA9525A21715A9222A95264211A
:1036D000715A29546820305A96216852B08E0C993C
:1036E0006852F08E0A996852308F08996852708F2C
:1036F0009E216852B08F0B996852F08FA2216852B8
:103700004020305A099968524220305AA621685206
:103710004420305A0E9968524620305AAA216852E5
:103720004820305A0D9968524A20305AAE216852CA
:103730004C20305AB02168524E20305AB221685283
:103740006A20305AB42168526C20305AB62168522F
:103750006E20305AB82168527020305ABA2168520F
:103760003046C830416EBC22A950816EC022A9509B
:10377000C16EC422A950016FC822A9507221715A8A
:10378000CC22A952016ED022A950016B0E91416B3F
:103790000D91436C846C876FC06F0C902920C00022
:1037A0003158301840680E9A2A660D9A6A66AB66E0
:1037B000EC662F670C9A6A67A967E867A868401CDF
:1037C000D8216960A860392028700F98002804D09B
:1037D000794806F0A9F87068E860784C60680028BD
:1037E00006D5204608387649016076490160606850
:1037F000754E3068012739040F912168C9031FD421
:103800002168724A531C2360114202D12168490386
:1038100069D46068C00702D06068B84360606C48D3
:1038200007706C4C20686C490F700006400E401EFB
:103830006A49086010A8FDF7B5F8002820D0FEE717
:103840007D21C9003268121A8A42E2D222680F9B97
:103850001A42D5D03268121A8A42DAD222681A4243
:10386000CED03268121A8A42D3D222681A42C7D006
:103870003268121A8A42CCD222681A42E2D1BFE7D9
:103880000E9720680006800B554FC419FF20860252
:103890000CCD2046083DFCF7F7FE0028FED14D4830
:1038A0000068800230403818D4300835083484422B
:1038B000EED3454D2868414C21680F9A11420E9E67
:1038C00034D12168414A531C2360114202D121683E
:1038D00049034BD4F0076168014361606068FFF7FA
:1038E0000DF911B0F0BDB9047D22D20033681B1A66
:1038F00093428ED223680B428BD033681B1A9342BB
:1039000087D223680B4284D033681B1A934200D3BA
:103910007FE723680B4200D17BE733681B1A934291
:1039200000D376E723680B42E0D172E77D21C9001E
:103930002A68121A8A42CDD222680F9B1A42C0D03E
:103940002A68121A8A42C5D222681A42B9D02A6855
:10395000121A8A42BED222681A42B2D02A68121AB9
:103960008A42B7D222681A42E2D1AAE7B1047D2284
:10397000D2002B681B1A9342ACD223680B42A9D009
:103980002B681B1A9342A5D223680B42A2D02B6846
:103990001B1A93429ED223680B429BD02B681B1AA2
:1039A000934297D223680B42E3D193E7D3C7000831
:1039B00028000020E003002008CA00081020024070
:1039C00023016745AB89EFCD24000020FA83000076
:1039D000940F0020E075FF1F900F0020600F002063
:0439E00000F8FF07E5
:1039E40010B5FFB083B0E349086A086A0869096939
:1039F4004424C1B2AA2904D0E0433322CC2904D000
:103A040004E05520C043332200E0D0430146563140
:103A1400049208D0C0B2CC2803D0BB2806D1F54804
:103A240002E0F54800E0F54805F07CFF6E94F44DA3
:103A3400DB35EF4C103C2068284020600126310221
:103A440020686291084320607D205D90C100ED48AC
:103A540000686C9106F0C4FF401E010E37076F9694
:103A6400B207119203223A92920763920029E64E1A
:103A740023D1E6494860E64A1068E64B1840639B48
:103A84001843106000208860072008601068E1492E
:103A94000840119908431060DF486F990170B06BBA
:103AA4000843B063B06B084074907498706B3843EB
:103AB4007063706B38407490749868973A9B59029D
:103AC400D64A1068509188430127B9024B91401897
:103AD40010601068629908431060706D18210143EA
:103AE4007165106828401060306838216A91084078
:103AF400102201466792514072681A400223739360
:103B04005A4089184A424A41B90365917197790626
:103B14006991314608396B910968C14F00282ED04C
:103B2400002A2CD10720C00281436B9A11601068CF
:103B3400629908431060BB4801686B9A12684B9BFA
:103B44001A4228D10268521A022A6FD86B9A126854
:103B54001A4220D10268521A022A67D86B9A126854
:103B64001A4218D10268521A022A5FD86B9A126854
:103B74001A4210D10268521A022ADED956E0311FC5
:103B84000A68A94B1A40659B1A430A6000280BD0A7
:103B94009C48006815E09C4D281F0168A24A11400A
:103BA400659A1143016032E00720C0026B9A1168E4
:103BB4008143116010688004410F9C48C8409149BA
:103BC400086095490E78002E119D00D135465D9907
:103BD400C90006F005FF401E8E49884226D88B494D
:103BE40048608B4A10688B4B1840639B18431060E5
:103BF4000020886007200860002E17D0114608684E
:103C0400844A104028430860834806707E4D286823
:103C14006A9A1040202801D000F0FBFC686D2868E7
:103C24001040102801D000F0D1FD68687198C003DD
:103C3400389020684007800F00D14EE20720729030
:103C44000003714B1968014319607949F1391A6805
:103C54000A401A606B990968699A114200D005E21A
:103C6400694B586B6899084007D1596B689A11439E
:103C74005963596B114074917499684F3968629A09
:103C840011433960719C21046091664E31686E9DC8
:103C94003A68629B1A4219D13268521A022A27D80A
:103CA4003A681A4212D13268521A022A20D83A6863
:103CB4001A420BD13268521A022A19D83A681A42A7
:103CC40004D13268521A022AE2D911E06C99E83917
:103CD4004D4A526D0A4021020A438A42554901D095
:103CE40000F0DAFC484B5A6D0A4062990A435A655F
:103CF4000028454E04D101200007716B8143716394
:103D04003A98C043F16C0140F164119A501EF16C71
:103D140001401143F164706860990843706046483B
:103D240005F000FEFDF780FD444F04243C60FDF7E0
:103D34007BFD52943C60719840057290301F6D90E9
:103D44000068669000213E4E3E4C08E00021709BC6
:103D540098003D4A1150591C802900D1C7E06D9A42
:103D640010680B46304908407093190240181060DF
:103D74000BE0C046102002400A6802430A607298B1
:103D84003249086073990229E1D13868042865D161
:103D9400012038603E21735C725D521E551EAA419B
:103DA400012B6F9B00D11346002B6E9DE7D102229D
:103DB400725472553168CB681343CB600A6A8243EC
:103DC4000A620A6A02430A62214A914205D0214AE0
:103DD400914202D0204A9142CED1609AD31D8A6882
:103DE4001A40062ACBD003049A42C8D0C4E7C0467E
:103DF4001020024091C4000876C40008ACC4000836
:103E040024FEFFFF200000200810024010E000E024
:103E140020ED00E0FFFFFF00840F00200070004051
:103E24008813000024000020FF80FFFF0024F4001A
:103E3400F0F1FFFFFFFCFFFF20C600086C0F00201D
:103E4400440E0020200F0020EC07002000E100E0D9
:103E54000004004000400140002C01403868032861
:103E6400739990D13868032800D06FE77298B349EA
:103E74000860BFF34F8FBFF36F8F3568E868022186
:103E84008843E860286A719B98432862286A2862FC
:103E9400286AAB4A104207D14B9844302A6A02423E
:103EA40002D12868984328603E2033546E983354D6
:103EB40052983860A3480268002A07D02068A24BB1
:103EC4001B681B03C0182060092A03D8501C9D4A94
:103ED40010600AE000219B4A11609C4A11600A218B
:103EE40006F07EFDA96A491C41436E9D4BE77F2085
:103EF40001026191669C0C406D9B1968944A1140C3
:103F040021431960401EFDD1709078907790914CB8
:103F1400E06A02210F910843E062E06A08407B9066
:103F24007B98E06A52990843E062E06A08407B901B
:103F34007B98E06A202173910843E062E06A0840BC
:103F44007B907B98E06A719E3043E062E06A304087
:103F54007B907B98F92047017F4807617F496298ED
:103F6400886276962120379000047590700227901D
:103F7400749074AD08462946FCF70AFF7098779050
:103F840076907596669774977348183864902946A6
:103F9400FCF7FEFE7696709F759740205E907490B5
:103FA4006F4810382946FCF7F3FE77977697759695
:103FB4006298749069482946FCF7EAFE77977696EA
:103FC400759673987490654829463D46FCF7E0FE63
:103FD400206B30432063206B304074907498FF2032
:103FE4000E9000025F4A1168814365980143116095
:103FF4005D48279901605D4C0720B1040702629A6D
:10400400121D5B4B23605C926260A5605B97E76066
:1040140025616661A161679AE26125626562A562B4
:104024000D90E062256365635D206D90205C320332
:1040340000280F9F0C92139100D19DE06D98275496
:1040440018681F465E9B98435F9738605A95599548
:10405400579556952F461346679851905891314677
:10406400284653955C9D54955593E1E01D46296877
:104074000222709211430523994329603D490D683A
:10408400344E36686A9A1640102E00D188E20E68C3
:10409400761BBE4200D9E3E52E4E36681640102E3C
:1040A40000D17DE20E68761BBE4200D9D8E5294EC8
:1040B40036681640102E00D172E20E68761BBE429E
:1040C40000D9CDE5234E36681640102E00D167E2A4
:1040D4000E68761BBE42D3D9C2E520680221014393
:1040E4000520814321602348016823680722134087
:1040F400022B00D1A2E503685B1ABB4200D9AFE5ED
:1041040023681340022B00D198E503685B1ABB4275
:1041140000D9A5E523681340022B00D18EE503687E
:104124005B1ABB4200D99BE523681340022B00D1E4
:1041340084E50268521ABA42D7D991E580E100E0D9
:10414400111100000C0F0020700F0020200F002020
:10415400FF80FFFF081002401800005000040050C8
:104164001008005008E400E000E100E0200D002009
:1041740000300140240000205C2000272754F4492B
:10418400886B10438863886B104074907498C86A75
:1041940001252843C862C86A28407B90789777979E
:1041A400769702205F907590E02074907B9874A9B4
:1041B400649E3046FCF7ECFD7F977E977D977C9557
:1041C40038987B907BA93046FCF7E2FD7398E1496F
:1041D40008606D985F992154226810685E9988433D
:1041E4001060E802E36818430F210902884200D0F6
:1041F400A7625F925B9883425C9D00D80C9F5597A1
:10420400D548F13003405B93606B5A9020461030E0
:1042140007C85892E2695192226A5692626A599288
:10422400A26A579262685492A2685392719E709FD8
:10423400549A2A40C94DAD1D539B1D40AA180F9B8B
:104244001840104331400143589D2846279A104096
:1042540008436A99519B0B40034380200990569A66
:1042640002401A436698E030669057990140114322
:104274005F9B19605B9A55980243280C5299084039
:1042840010435999679D2940014308225A981040C8
:1042940008435860F002D9698143D96127666D9853
:1042A40026543C20AE4C129026542C206D9026545B
:1042B400256473986064A764E76427630D9860635A
:1042C400A0636762A762E661A6762783A54D201DD9
:1042D4000777A548183025606060A760E7600790FD
:1042E4002061359262617D977C977B978097A06D62
:1042F400002805D0A868689F384200D1A7E0CEE026
:1043040000247894779401231805914A916B014312
:104314009163916B014081918198D06A1843D06276
:10432400D06A1840709381908198D06A022171916B
:104334000843D062D06A084081908198769403271C
:104344007597749374AD649E30462946FCF720FD3E
:10435400769475977198749030462946FCF718FD49
:104364007694759704206790749030462946FCF73C
:104374000FFD76947597709874907C48064629468C
:10438400FCF706FD7694759771987490304629462B
:10439400FCF7FEFC7694759767987490304629462E
:1043A400FCF7F6FC7694759735987490649E3046C5
:1043B4002946FCF7EDFC76947597102074903046EE
:1043C4002946FCF7E5FC25216948719A4254694A5B
:1043D4000F32694B1D6815401D604D2252011D6846
:1043E40015431D60654A05251560654F709E3E6046
:1043F400C46346540462F102802728C00460446008
:104404008760629BC3600161739941618463C26385
:104414008032026446648464C464046524210838D8
:1044240044544F4908658162564A50680E9988433E
:1044340050600C9854490860542049490C54484829
:10444400C465474C2568A868689F384227D1A86886
:104454004E4901403943A9604D4800684D4906F072
:10446400BFFA4000801C80908098002817D0809864
:10447400401E80908098002811D08098401E809023
:10448400809800280BD08098401E80908098002847
:1044940005D08098401E809080980028E7D1A868B5
:1044A40038423D4E07D1A06D10210143A165E06D56
:1044B40001210143E165A868529908401022A16DC9
:1044C400114008180F215B91C94364910028A16D24
:1044D400679239D13148D9300140022071900143AB
:1044E400A1652169AA68D20700D06DE2236B002B75
:1044F4000C9A00D100220029729B02DA1A4B17335E
:104504000B402646A4681C43337E9B032343747EDE
:10451400E4031C43B37E5F032743F4683C43144322
:104524006D98325C52002243739FF45D012C00D0DD
:1045340009E2002B00D104E20948836D3B43836503
:10454400C36D1C43C465FFE11143A165A0E2C046ED
:1045540008100240180000500F0E0000FA830000FB
:10456400840D002000240140E8FFFF7F0004005078
:10457400E80D00200080FFFF080002400008024010
:104584008408024008E400E000E100E0E8FFFF6F77
:1045940020000020400D03002400002024FEFFFF23
:1045A4002568729A1540032D00D2B7E02568709AE9
:1045B40015439D4325600A682368729D2B40022B96
:1045C40000D1ABE00B689B1ABB4201D9FFF748FB53
:1045D40023682B40022B00D1A0E00B689B1ABB423E
:1045E40001D9FFF73DFB23682B40022B00D195E056
:1045F4000B689B1ABB4201D9FFF732FB23682B409F
:10460400022B00D18AE00B689B1ABB42D4D9FFF776
:1046140027FB686B6899084007D1696B689A114356
:104624006963696B114074917499F4490968629AD9
:10463400114200D09EE0F14B196811431960FE4904
:104644000A68FC4B1B68629D2B4200D092E00B6809
:104654009B1A022B01D9FFF7E9FAF64B1B682B4290
:1046640000D087E00B689B1A022B01D9FFF7DEFA12
:10467400F04B1B682B427DD10B689B1A022B01D98E
:10468400FFF7D4FAEB4B1B682B4273D10B689B1AD0
:10469400022BD6D9FFF7CAFAE84F7A6D7B6D609C7E
:1046A40023437B657B6DA3437B6513460B407B658E
:1046B400E34CD20701D1FFF715FB3268DF4B5B6D8A
:1046C4009B0701D5FFF70EFB33689B1AA34201D960
:1046D400FFF70EFBD94B5B6D9B0701D5FFF702FB80
:1046E40033689B1AA34201D9FFF702FBD34B5B6DDE
:1046F4009B0701D5FFF7F6FA33689B1AA34201D949
:10470400FFF7F6FACD4B5B6D9B0701D5FFF7EAFA8D
:1047140033689B1AA342D1D9FFF7EAFAC74C216840
:104724008143216020688006400F00D1CEE02068DC
:104734006A9A10400828C34800D1CDE0216811408E
:10474400102901D001F081F8616803220A40032A8C
:1047540000D0BD4861684906490F491C06F040F97C
:1047640061684904490E48436168490F491C06F0D1
:1047740037F9B1E0B14A516D719B19435165AE49A6
:104784000A68AE4D6B6D9B0751D40B689B1ABB42F4
:1047940001D9FFF74BFA6B6D9B0748D40B689B1A42
:1047A400BB4201D9FFF742FA6B6D9B073FD40B68FC
:1047B4009B1ABB4201D9FFF739FA6B6D9B0736D4BC
:1047C4000B689B1ABB42DCD9FFF730FA71980006DC
:1047D4006B9A116881431160974801686B9A12685B
:1047E400699B1A422FD00268521A022A01D9FFF794
:1047F4001DFA6B9A12681A4225D00268521A022ACC
:1048040001D9FFF713FA6B9A12681A421BD0026897
:10481400521A022A01D9FFF709FA6B9A12681A424E
:1048240011D00268521A022AD8D9FFF7FFF90028DA
:104834006A9A01D0FFF7F3F971980007696B814315
:104844006963FFF7ECF97D4B5968804A0A40804957
:10485400511859607F49491C6B9D2A680A432A6094
:104864005968689A1143596001686B9A1268699B88
:104874001A4201D0FFF7DAF90268521A022A01D962
:10488400FFF7D4F96B9A12681A4201D0FFF7CEF9F8
:104894000268521A022A01D9FFF7C8F96B9A126802
:1048A4001A4201D0FFF7C2F90268521A022A01D94A
:1048B400FFF7BCF96B9A12681A4201D0FFF7B6F9F8
:1048C4000268521A022AD0D9FFF7B0F96B9800682F
:1048D4008004410F5C48C840216889093C220A4091
:1048E4005D4989581F220A40D0405C4908605C4CED
:1048F4002578002D119E00D12E465D99C90006F041
:104904006FF8401E5349884201D9FFF7A9F9554968
:104914004860554A10684F4B1840639B1843106019
:104924000020886072980860002D01D1FFF798F983
:1049340011460868474A1040304308602570FFF765
:104944008FF9609B1A434948436A876AEE68484C6A
:104954003440002B709103D0629EC03633403B43F9
:1049640013432343EB60426863991140C36C129C68
:10497400045D012C09D1046C466C2643846C3443D9
:104984000C431C430121214300E019432A4E2B69A7
:10499400384C1C400C432C610123DC07A242334CED
:1049A400709911D00324A407A242304C0CD09B0769
:1049B4009A4209D05B9B9B041A402F4C26689E4365
:1049C400B2181D4E2260294C6A690D9B9A43636B91
:1049D4001A436A616A6920467024A243846B2401E5
:1049E40014436C6101225405A14209D0002913D15A
:1049F400A96A64980143A9620EE0C04600700040B1
:104A0400A96A1A48C16989001C311C240C406499A4
:104A1400A140046E0C43AC6269690D9C214099422B
:104A24002CD100211148C165816D1143719A9143C4
:104A340081652DE000700040240000200810024031
:104A44008813000000127A000024F4008C80C11F37
:104A540002080220FFFFFF0090BB00082000002096
:104A6400840F002010E000E020ED00E0840D002021
:104A74000102DEFF02FCFF1F08270140FC4CA16D70
:104A840010230B4371988343A365E06D1043E065E5
:104A940000277D9701247C947B947BAD2846FBF70B
:104AA400CFFBA0061890801C7B902846FBF7C8FB20
:104AB4006D94E0065C90001D7B902846FBF7C0FBDC
:104AC400EC487B902846FBF7BBFB689810307B9042
:104AD4002846FBF7B5FBE8487B902846FBF7B0FB7C
:104AE400E6487B902846FBF7ABFBE5487B902846DD
:104AF400FBF7A6FBE3487B902846FBF7A1FBE24CBF
:104B04007F20A7605790E0600E9820616761A761DD
:104B1400E7611198206271976762DC4802460C3A9B
:104B240022602927E15D002912D128210023635442
:104B34001121C9026160D64D696B4B9B19436963AE
:104B4400696B194074917499696D389B194369654F
:104B54000F990697E155CA215A91816153218161C8
:104B640003685B066D9F27D4036880241C4304609C
:104B74003368046864061FD43468E41A6C9DAC423C
:104B840014D80468640617D43468E41AAC420DD807
:104B94000468640610D43468E41AAC4206D8046885
:104BA400640609D43468E41AAC42E2D90323B64C4F
:104BB400069D6355036868E0C368B64C1C40C46036
:104BC400C368C3600E9B4360579B1B0444681C432B
:104BD40044600368099CA3430360C3689B0626D40E
:104BE4000368A024A343036033680468A40654D470
:104BF4003468E41A6C9DAC4214D80468A4064CD4FE
:104C04003468E41AAC420DD80468A40645D4346868
:104C1400E41AAC4206D80468A4063ED43468E41A04
:104C2400AC42E2D93A9B984C069D63552DE0C3688B
:104C3400739CA343C3600368A024A3430360336845
:104C44000468A40625D43468E41A6C9DAC4214D8D4
:104C54000468A4061DD43468E41AAC420DD8046870
:104C6400A40616D43468E41AAC4206D80468A40630
:104C74000FD43468E41AAC42E2D93A9B824C069DC4
:104C84006355C368739C2343C3600E9B83617E4B4F
:104C940011E0C368739C2343C360C3687C07641E2C
:104CA4001C40C460C368119C2343C3600E9B836192
:104CB400754B069C1F5528240B941B5D012B00D1BA
:104CC4005AE10F9B704C069D63550B9BE7545A9B0E
:104CD4008361816103685B0627D40368099C2343CD
:104CE40003603368046864061FD43468E41A6C9D56
:104CF400AC4214D80468640617D43468E41AAC428D
:104D04000DD80468640610D43468E41AAC4206D89A
:104D14000468640609D43468E41AAC42E2D93A9AC5
:104D2400594B069D5A55026864E0C3687B041360BE
:104D3400BA04C3689343C360C268C2600268099B33
:104D44009A430260C268920626D40268A0239A435A
:104D54000260326803689B0653D433689B1A6C9CC8
:104D6400A34214D803689B064BD433689B1AA3420E
:104D74000DD803689B0644D433689B1AA34206D813
:104D840003689B063DD433689B1AA342E2D93A9A3E
:104D94003D4B069D5A552DE0C268739B9A43C260F1
:104DA4000268A0239A430260326803689B0624D4F5
:104DB40033689B1A6C9CA34214D803689B061CD4CA
:104DC40033689B1AA3420DD803689B0615D4336835
:104DD4009B1AA34206D803689B060ED433689B1A19
:104DE400A342E2D93A9A284B069D5A55C268739C4D
:104DF4002243C2600E9A826108E0C268739B1A4320
:104E0400C2600E9A8261204B069D5F550F9A5A55D7
:104E14000B9A9F545A9A82618161016849063BD476
:104E24000168099A1143016031680268520633D45B
:104E34003268521A6C9B9A4214D8026852062BD4D8
:104E44003268521A9A420DD80268520624D4326843
:104E5400521A9A4206D8026852061DD43268521A6F
:104E64009A42E2D93A99084A069BD154016873E000
:104E7400840D00200800000C001000B00001002088
:104E84000002002400040028900E00200C2800409A
:104E940008100240BFFF8FFB01460839B44A0A607C
:104EA4000168099A91430160C168890626D40168A2
:104EB400A0229143016031680268920654D432689A
:104EC400521A6C9B9A4214D8026892064CD43268E7
:104ED400521A9A420DD80268920645D43268521A80
:104EE4009A4206D8026892063ED43268521A9A420E
:104EF400E2D93A999F4A069BD1542DE0C168739A2E
:104F04009143C1600168A022914301603168026845
:104F1400920625D43268521A6C9B9A4214D80268BD
:104F240092061DD43268521A9A420DD8026892062B
:104F340016D43268521A9A4206D8026892060FD4DE
:104F44003268521A9A42E2D93A998A4A069BD15453
:104F5400C168739B1943C1600E998161104608E0D2
:104F6400C168739A1143C1600E99816181480699A1
:104F740047540B99719A4254F74D286B0C9B184374
:104F84002863F64C27620D9AA260679DE5600E982F
:104F94002061719F6761A7610230A080F5480146D6
:104FA40008392160EC49096B194074917499617F47
:104FB400002900D121770F9B6377C26001682943E0
:104FC400359A9143016021698160016860229143AF
:104FD40001600168099A914301606D9D657728021B
:104FE4005590FF30E44A10801446C834E765A7653D
:104FF40045204A908100F8430591505264990F313D
:105004006164A164472116918900159150528F2142
:105014004900149150522321C900089150528D2106
:105024004900029150521381558105203690908198
:1050340007982062D148173059906062D048208187
:10504400411E5491618160616198FF30A061C1206B
:1050540040002D901752106ECA4B58430699C90050
:105064005050649151186391C0174860D06D5843F3
:10507400A067C0177094E067C348806B0006800B7C
:10508400C249405C382815D0392809D0FF281DD1E1
:10509400BF4804F047FCB8494F800E98C88118E017
:1050A400BC4804F03FFCB4494D803920C881FDF769
:1050B40023FD10E0B84804F035FC0220AE494880D6
:1050C4006A98C8810020FDF7DBFE04E03A9951801C
:1050D400D081FDF76FFBB14804F024FCFDF70CFD13
:1050E400AF48006840061AD430683168091A32297A
:1050F4000BD83168091A322907D83168091A3229BC
:1051040003D83168091A3329EFD3A548006840064B
:1051140005D4A44804F006FC0120FDF7B1FEA24822
:10512400A24A02600C24A24B54619761D7611762B2
:10513400576297629049086913605060888A9D4A53
:10514400531EC98ACA1E92B210939A422A4600D3A9
:105154000A46022801D3092100E00A2192B200285C
:105164004B9D0C9B0AD0012806D1509D06E0C046F9
:1051740016241800900E00203D463B4688188B49A3
:1051840061938B605F950D61012A00D0669F874D06
:105194006697EF6005F09AFB874B719F3A4606F0DD
:1051A40033FE05F00BFB5890099AA85800283E4698
:1051B40038463B4639467E4F41D17C2000247B490A
:1051C4000C546549886B659A10438863886B10405A
:1051D40074907498C86A02252843C862C86A284033
:1051E4007B90789477940120769075955E9874906E
:1051F4007B9874AE714F38463146FBF7C9FD7894FD
:105204007794769475958020749038463146FBF7F0
:10521400BFFD099A6A4B18696A49084018616A48CF
:105224005C990160614DA8686190E868669028699E
:105234005F906C69AB69E969286A6E6A2F685C9350
:105244000B4624215691594DA9503A680121539196
:105254008A433A605F990C4361990C436A6E224316
:105264003C685A4D2540154365931D433D603A9A69
:1052740012037C68944366990C437C605C990843F0
:10528400BA68534B13400343BB60F86A5B9A90437C
:105294003043F8624F4887423B46354609DC4E4866
:1052A40083424E4E679917D04D4883423F4F1BD0DF
:1052B40010E04C488342494E3C4F679914D03C4817
:1052C400834207D12448C06C8007000F464A105817
:1052D400719009E0719107E01F48C06C0C220240F4
:1052E400414880587190314F67936D98C003389A44
:1052F4006599914226D17199082900D959E149004B
:105304007944898849008F4408005401D800540125
:105314008A00540154015401E400344800680E49E1
:105324000968890A1C220A40314989581F220A4007
:10533400D0400B2D00D2F8E00B2D629900D1F7E09C
:105344000121F5E07199082900D932E104A249004C
:10535400515A49008F44C04608100240BC0E002038
:105364004E002D01B7002D018A002D012D012D01C4
:10537400C300C0460830024028000020E8FFFF7F39
:105384000080FFFFF0F1FFFFA875FF1F00F8FF0783
:105394000AC6000891C70008EEC3000854C40008F8
:1053A4001008005063C40008B8050020940A0020C7
:1053B40000380140FFFF000000000C4000040050D2
:1053C40008E400E0FFFFFF0000E100E0F369FFCF25
:1053D400FFF4FF11FF4B0040004400402400002074
:1053E40000480040004C004054BB0008200000204E
:1053F400D0BB0008F9480068F9490968890A1C22E9
:105404000A40F84989581F220A40D0400B2D00D287
:10541400A8E00B2D629900D1A7E00121A5E0F04A94
:1054240010688006400F77D010686A9B18400828DF
:10543400ED4877D011681940102900D014E2516862
:1054440003220A40032A00D0E848E54C6168490673
:10545400490F491C05F0C4FA61684904490E4843E0
:105464006168490F491C05F0BBFA5BE0DC4A10682F
:105474008006400F6DD010686A9B18400828DA48EF
:105484006DD011681940102900D0FAE151683A9A98
:105494001140032900D0D548D14C61684906490F11
:1054A400491C05F09DFA61684904490E4843616846
:1054B400490F491C05F094FA51E00B2D15D2A800B0
:1054C400CB49095814E00B2D14D2A800C849095837
:1054D40013E00B2D13D26900C64A515A12E00B2D6A
:1054E40016D26900C34A515A3FE0629900D00121A3
:1054F400BE481DE0629900D00121BC4835E05599B1
:1055040000D0012105F06CFA41007C68600814E0C9
:1055140055992AD0539928E06B9800688004410F6C
:10552400B248C8400B2D00D306E7A900B04A515831
:1055340005F056FA40007C6861080818214605F019
:105544004FFA60991039014033D00007400F0843E7
:1055540016E06B9800688004410FA448C8400B2DE6
:1055640000D356E7A900A24A515805F039FA7C68DD
:1055740061080818214605F033FA80B20F2818D9BB
:10558400679AD06000259C48B866FD663D67B86A96
:10559400002870D0C10713D181071BD4410723D43D
:1055A40001072BD4C10632D481063AD4410642D431
:1055B40057E09148B8660020F8663867739FD9E0D1
:1055C40001214904134652688A43F96A1143596018
:1055D4008107E3D501210904679B5A688A43396B23
:1055E400114359604107DBD501218904679B5A683F
:1055F4008A43796B114359600107D3D5679B596876
:10560400549A1140BA6B0A435A60C106CCD50121A1
:105614000903679B9A688A43F96B11439960810671
:10562400C4D501214903679B9A688A43396C1143A5
:105634009960410615D50121090571953546679E86
:1056440072688A437B6C1A4372602E46719D8B424A
:1056540007D13A994905679B5A688A43B96C114343
:1056640059600006679A06D50120C0045168814339
:10567400F86C084350600127F805516801435160F4
:1056840010681899084310603A984002D630604375
:105694005A4905F0A5F95A498C42589A00D3421C3C
:1056A4005848401C679C616901401143616120684E
:1056B40038432060882054490D5030682168090718
:1056C40022D5E169729A11421ED131680A1A699988
:1056D400491E8A423ED8E269729B1A4214D132684A
:1056E400121A8A4236D8E2691A420DD13268121A65
:1056F4008A422FD8E2691A4206D13268121A8A42C3
:1057040028D8E1691942E0D0216849072AD5E1691E
:10571400490227D4B9053268131A699A521E934272
:1057240018D8E3690B421DD133681B1A934211D870
:10573400E3690B4216D133681B1A93420AD8E36912
:105744000B420FD133681B1A934203D8E2690A4211
:10575400E1D007E02D483B30216801402160A0687A
:10576400B843A06009982849739F0F507C200D54BA
:1057740084200F50264800687C210A91445C01462D
:105784007C31012C0ED0569A4A6002681368156861
:105794000126B54315607507AB43136000224266CA
:1057A4000A704F608A68202A0C9E13D103465C332A
:1057B4008268B2420CD1012C0CD00469002C09D0AF
:1057C400559C5C801C800E9C9C80124C846567E018
:1057D400012C23D1104805F0CFF9FEE7200000206A
:1057E40008100240D0BB000800127A000024F40024
:1057F40064BB000834C100080100010040420F00EE
:10580400014B0000FFFFFFFE940A002024FEFFFF6F
:10581400B8050020DF05002094C50008559C5C8075
:105824001C80FD4C8465002A08D001242407A24270
:1058340009D10469002C04D03F2430E00469002C11
:105844002CD0579C2BE0002429E02068104020280D
:10585400389801D1FFF740F820681040182800D18B
:10586400A3E10020FFF738F8106818402028389882
:1058740000D157E610681840182800D1CEE1002066
:1058840050E6106818402028389800D167E6106860
:105894001840182800D1C4E1002060E60E9C9C80CA
:1058A40000247394CC60222439948C600468A56825
:1058B40001273D43A56058977F07456E0197BD4278
:1058C40003D19B89559DAB420ED9B24203D10269E3
:1058D400002A00D1CEE0D44AD44E00230B70C26615
:1058E400629F2037224611E0B24203D10269002AA6
:1058F40000D125E1CE4BCD4E689F224608320025CB
:105904000D70C36620686299084320602620659064
:10591400739D3554106838431060F561B58435843F
:1059240030461C308571C34F388804F0BFFF7321A3
:10593400CC05214604F082FDBF4F394604F07EFDBC
:1059440004F02AFF0646BD480660BA48408C04F0BD
:10595400ADFF214604F072FD394604F06FFD04F0FA
:105964001BFF801BB649086054277495B54BD85D5E
:105974005899CA05039201281C68349702D1A0687B
:10598400B14EE4E2D955A068A168C907AE4E23D050
:105994000F99084020D1A06836990840012812D1F7
:1059A400A068AA4908400F990843A0603A9820606B
:1059B4003068A168C9070FD03168091A0329F8D3E0
:1059C400A168C907F5D09F4A906D102101439165E4
:1059D400D06D58990843D065A068C007994A906D66
:1059E40040D19B49D93108400F9908439065E1683B
:1059F4009848001FE2680240E260A068934A1040A1
:105A040010181830A0603898C01C084072902146C5
:105A1400B431914AA368002B2ED5749B5B1C7493FC
:105A2400749B934200D9B5E1A368002B24D5749BE1
:105A34005B1C7493749B934200D9ABE1A368002B65
:105A44001AD5749B5B1C7493749B934200D9A1E197
:105A5400A368002B10D5749B5B1C7493749B9342B6
:105A6400D8D997E1102108437649739ACA558865B5
:105A7400104698E1794A2FE70B68A56873480540FA
:105A840045191835A56057980340A568002D24D5FD
:105A9400749D6D1C7495749D954200D97AE1A56836
:105AA400002D1AD5749D6D1C7495749D954200D972
:105AB40070E1A568002D10D5749D6D1C7495749DBE
:105AC400954200D966E1A568002D06D5749D6D1C2C
:105AD4007495749D9542D8D95CE10D68A6685B48BD
:105AE400064086191836A660574E57980540EB189D
:105AF400A568002D26D5749D6D1C7495749D9542E2
:105B040000D947E1A568002D1CD5749D6D1C7495C2
:105B1400749D954200D93DE1A568002D12D5749D70
:105B24006D1C7495749D954200D933E1A568002DD0
:105B340008D5749D6D1C7495749D9542D8D929E13E
:105B4400474BD8E60D68A6684048064086191836C3
:105B5400A6603D4E579805405B19A568002D28D5D1
:105B6400749D6D1C7495749D954200D912E1A568CD
:105B7400002D1ED5749D6D1C7495749D954200D99D
:105B840008E1A568002D14D5749D6D1C7495749D51
:105B9400954200D9FEE0A568002D0AD5749D6D1CC0
:105BA4007495749D9542D8D9F4E05D980002FEF78F
:105BB40093FE0D68A6682548064086191836A66027
:105BC400214E579805405B19A568002D4AD5749D50
:105BD4006D1C7495749D954200D9DBE0A568002D79
:105BE40040D5749D6D1C7495749D954200D9D1E087
:105BF400A568002D36D5749D6D1C7495749D9542D1
:105C040000D9C7E0A568002D2CD5749D6D1C749532
:105C1400749D9542D8D9BDE0DF0500205D9800024F
:105C240080E45D9800029AE451BD0008B8050020A4
:105C3400F1130008A875FF1F00803B45280F0020C2
:105C4400240F0020840D002024000020E8FFFF7FA3
:105C540024FEFFFF0080FFFFFFF1020097C1000850
:105C6400291600080D68A668E84806408619183603
:105C7400A660E74E579805405B19A568002D22D50C
:105C8400749D6D1C7495749D954200D982E0A5683D
:105C9400002D18D5749D6D1C7495749D954279D80A
:105CA400A568002D0FD5749D6D1C7495749D954247
:105CB40070D8A568002D06D5749D6D1C7495749DCF
:105CC4009542DAD966E00D68A668D0480640861980
:105CD4001836A660CE4E579805405B19A568002D6E
:105CE40021D5749D6D1C7495749D954252D8A568F8
:105CF400002D18D5749D6D1C7495749D954249D8DA
:105D0400A568002D0FD5749D6D1C7495749D9542E6
:105D140040D8A568002D06D5749D6D1C7495749D9E
:105D24009542DBD936E00D68A668B8480640861966
:105D34001836A660B64E579805405819A568002D28
:105D440001D403F023F8749D6D1C7495749D9542E1
:105D540020D8A568002D01D403F018F8749D6D1C9B
:105D64007495749D954215D8A568002D01D403F04F
:105D74000DF8749D6D1C7495749D95420AD8A568A0
:105D8400002D01D403F002F8749D6D1C7495749D6C
:105D94009542D3D900209F4BD855996D10220A43C0
:105DA4000F998A439A65411E48424841A1684907B0
:105DB4006F9900D40146002900D0C8E0589995484D
:105DC400C155E068C0070CD1A068C00706D0A06820
:105DD4008E4908400F9908435899A060E068084329
:105DE400E06073987490A068C00741D187482F3051
:105DF400A168014209D0874A906D10210143916541
:105E0400D06D58990843D065A1E0A0687F49084047
:105E140058990843A060804800680399084221D03B
:105E24007E4800687E4904F0DBFD401C7490749841
:105E3400002817D07498401E74907498002811D0CC
:105E44007498401E7490749800280BD07498401E67
:105E540074907498002805D07498401E74907498B7
:105E64000028E7D16B48407E012801D002F074FF7E
:105E7400684A739BD3556B48FF30916D014062981B
:105E840001439165D3651C232360106D6649674AFD
:105E9400674DC56202634163616810220A43626010
:105EA4005699415C01294CD001462431589D0D700E
:105EB4004A78012A41D10F9A4A707399C1630168E3
:105EC4000A68AA430A60826CC56C5560026D002A98
:105ED40002D0456D866D6E6025464035066C1E40C9
:105EE400589BB340534E361F37681F43376009230E
:105EF4004B608668504B102E1F4600D02F468F6093
:105F0400102E00D01D46CD600B680E251D430D607C
:105F1400406C0368609D2B423D4E03D00368629D34
:105F24002B430360002A03D01068629B184310605F
:105F34000868589A1043086003E0739A0A70099934
:105F4400C163A0683149084052990843A060306891
:105F54003168091A64290BD83168091A642907D8E9
:105F64003168091A642903D83168091A6529EFD3FD
:105F7400FBF778FD314803F0D5FC70983049C187B0
:105F84008187304F388B002831D05898C0020021C7
:105F940004E0491C2B4A128B914228D22A4A1060F1
:105FA40033683268D41A629A5E3294420BD83468E9
:105FB400E41A944207D83468E41A944203D8346843
:105FC400E41A9442EDD9204B186133683468E41A1A
:105FD4009442DED83468E41A9442DAD83468E41A75
:105FE4009442D6D83468E41A9442EFD9D1E7E12038
:105FF40000016B904D20179040010021134D5F303C
:1060040019906D9169915F912BE0C046E8FFFF7F85
:1060140024000020840D00200827014020000020D7
:10602400400D0300FFEFFFFF4BC10008FDBC00085B
:10603400D101000808000240E00E0020E8C7000873
:10604400FFFF0000280000201800005001A00000FD
:10605400002073997050307584209249399A0A50FF
:1060640039466A9190480068012801D000F0F8FB95
:1060740000258D4805608D4F38688109401A8C4F82
:10608400B9684418A1098B484843000CC8228A4BBC
:1060940098528A4804F0A4FC709E70803868C11736
:1060A4007288002304F05CFC0622002304F058FCF0
:1060B4000904000C4018F0607C48046080480068C3
:1060C4007C6880491731739188426F9908D0411CCC
:1060D4007B4A11601999884201DC002100E001210A
:1060E4007291794A1068010A401A00191060000A76
:1060F400718800230A0C050C2F46574380B2424393
:106104008EB270436E43150C110440187D41310C5E
:106114003204709E10186941062204F021FC09041F
:10612400000C40183061729800280BD030697169F6
:10613400884201DD306970613069B169884201DAF1
:106144003069B0615A985C4E305A0025210C020C1B
:1061540013464B4380B24143A4B2604354430A0CF8
:10616400090440185A41210C2304181851410622ED
:106174002B4604F0F5FB0904000C40186521890046
:1061840070504B49C868514A12680969739B9A4216
:1061940002D0521C4D4B1A60401A04F04BFB0446CB
:1061A4000E46709F788804F091FB2246334605F032
:1061B4002BFE2A46464B05F027FE2A46454B04F0A3
:1061C40099F9454A454B04F095F904460E46942046
:1061D4003949085804F02EFB2A46414B04F08AF949
:1061E4002246334605F010FE04F082FA19210A0112
:1061F4007292314988503A69D317F869C11704F08B
:10620400AFFB5D9AD2002B4604F00EFC386435488F
:106214000068396E081ACD214900274A5052324984
:10622400081D7C2205F05CFC304E301D31467C227A
:1062340005F056FC72982049085872902A49086063
:10624400F868539030602A462B46739806E02D1D5B
:10625400802D73913A463346204619D02349495933
:10626400CC176140091B91420F4600DC1746739A14
:10627400914200DB11461C4A5259D4176240141B48
:106284009C42264600DC1E468442E0DB0446DEE7F0
:10629400781AC1174840401A5190642828D3002521
:1062A40027E0C046940A0020080F00204C0F00206D
:1062B400E00E0020E40C0000280000200000B80BD1
:1062C400740F0020E8FFFF7F780F00205C0F002090
:1062D4000000F03E00004440FCA9F1D24D62303F82
:1062E40080842E41640F0020200C0020200B00200D
:1062F4000125094F301BC1174840441AF86D682125
:10630400795A04F06DFBC117890F4018801050941E
:1063140084426F9803DB01E028000020284600280F
:10632400014D03D09CE2C04601A00000074842682A
:106334008368981AC1174840401A72992492511AD6
:10634400CA175140891A884203DC01E0200C00205E
:1063540008460449CC68E11ACA175140891A814297
:1063640003DC01E0200C0020014604480569281BD9
:10637400C2175040801A884203DC01E0200C002040
:10638400084604494E69711BCA175140891A814253
:1063940003DC01E0200C0020014604488769B81B97
:1063A400C2175040801A884203DC01E0200C002010
:1063B40008460549C9694F91C91BCA175140891A32
:1063C400814204DC02E0C046200C0020014605485E
:1063D400026A4F984E92101AC2175040801A88428F
:1063E40003DC01E0200C0020084605494A6A4E9966
:1063F4004D92511ACA175140891A814203DC01E0B7
:10640400200C002001460548826A4D984C92101ACF
:10641400C2175040801A884203DC01E0200C00209F
:1064240008460549CA6A4C994992511ACA175140FB
:10643400891A814203DC01E0200C00200146054852
:10644400026B49984892101AC2175040801A884229
:1064540003DC01E0200C0020084605494A6B4899FA
:106464004792511ACA175140891A814203DC01E04C
:10647400200C002001460548826B47984692101A6A
:10648400C2175040801A884203DC01E0200C00202F
:1064940008460549CA6B46994592511ACA17514094
:1064A400891A814203DC01E0200C00200146FE48E9
:1064B400026C45984492101AC2175040801A8842C0
:1064C40000DC08465490F848426C4498101AC117EE
:1064D4004840411A54988142269100DC0146559166
:1064E400F148806C4390801AC1174840411A55986E
:1064F4008142289100DC01465691EB48C16C4398D7
:106504004291081AC1174840411A5698814229916C
:1065140000DC01465791E448016D42984191081A04
:10652400C1174840411A579881422A9100DC01461C
:106534005C91DD48416D41984091081AC11748406B
:10654400411A5C9881422B9100DC01466191D64846
:10655400816D40983F91081AC1174840411A6198CB
:1065640081422C9100DC01466691CF48C16D3F9871
:106574003E91081AC1174840411A669881422E91EB
:1065840000DC014620976791C748016E3E983D9113
:10659400081AC1174840411A679881422F9100DCBC
:1065A40001462F466891C048416E3D983C91081AB7
:1065B400C1174840411A68988142309100DC014675
:1065C40025467191B848816E3C983B91081AC117D1
:1065D4004840411A71988142319100DC014673911F
:1065E4001F922196B048C26E3B98101AC1174840BA
:1065F400441A73988442329400DC04462593AA48D2
:10660400036F1E92991ACA1751408E1AA642314638
:1066140000DC214633942395446F1D93E21AD3176B
:106624005A40D31A8B421A4600DC0A462297856FD9
:106634001C942C1BE7177C40E41B9442274600DC87
:106644001746C06F1B951A90401BC5176840401B26
:10665400B842964D00D903E1944200D900E18B423F
:1066640000D9FDE03398864200D9F9E07398329955
:10667400814200D9F4E071983199814200D9EFE068
:1066840068983099814200D9EAE067982F9981424D
:1066940000D9E5E066982E99814200D9E0E061983E
:1066A4002C99814200D9DBE05C982B99814200D976
:1066B400D6E057982A99814200D9D1E05698299971
:1066C400814200D9CCE055982899814200D9C7E08D
:1066D40054982699814200D8C2E0519804F0AAF84F
:1066E40004460D46509804F0A5F802460B46204691
:1066F400294603F0FFFE00226D4B05F085FB03F0F5
:10670400F7FF14996B4B58522520C000185871900C
:106714005720C000739019187298C8676722D00078
:1067240072901B185398D86724988867624A151D7D
:10673400E0CD10695469619494696694D46967944E
:10674400146A68949D67259D4D675E67239D0D6758
:106754001F67229DCD66D8662198886661989866E1
:106764005648719C046020984866669858664F980D
:106774000866679818664E98C8656898D8654D98F5
:106784008865506A946AD56A166B576B6697976BDF
:106794006797D76B6897176C719798654C9848659D
:1067A4005C65499808651D654898C864DE64479827
:1067B40088646698986446984864679858644598CD
:1067C4000864689818644498C863DF631F988863F2
:1067D400506C946CD56C166D576D6697976D679772
:1067E400D76D6897176E71979863439848635C6395
:1067F400429808631D634198C862DE6240988862CB
:10680400669898623F984862679858623E98086212
:10681400689818623D98C861DF613C988861506E41
:10682400946ED56E166F576F6897976F7197D26F86
:1068340098613B9848615C611E9808611D611D98D0
:10684400C860DE60194D1C988860689898601B9831
:1068540048605F60174F1A987399785072983A504D
:1068640017480068012801D000F0CEFC74A800216C
:1068740001720226134B5E77186882680124224352
:1068840082607591104A74921A6A012A20D0022AF1
:1068940006D0032A0A461ED10B4A0260002200E0F9
:1068A4000A4A026016E0C046200C002001A0000045
:1068B40000408F4028000020200B0020640F00209F
:1068C400040F0020BC0E002012EC0000000012ECAB
:1068D400C64A0280026874A88270C54A73945477C9
:1068E4007BAC21727C917B91389FC24D2F61092230
:1068F4002146FAF7E9FB2F602078FF28BE4D5AD1D4
:1069040074A800787BA94978814254D174A840784E
:106914007BA9897881424ED174A880787BA9C978F3
:10692400814248D12F46B24D6E777BA8007A2A68FF
:10693400936801210B4393602B6A012B17D0022B20
:106944000AD0032B1CD17C9B13607D9B13607BAB13
:10695400DC6814601B690CE07BABDC887C9E36042D
:10696400341914605B897D9C2404E31801E07C9B4A
:106974001BBA13601268697782423D4605D01AE05B
:106984000022697782423D4615D17BA80079CC214B
:10699400014084290FD17BA841790904827912022C
:1069A4005118C07908180399491E88420AD9934995
:1069B4000818801C06E02D99685A401C6852FBF7A1
:1069C40051F800208E490968599A91426F9A07D06C
:1069D4004A1C8B4B1A60132901DC00217391739AB2
:1069E4007292884909680818CA0F89184910441A0C
:1069F400E00F201847103120C0002F50A86F73906B
:106A0400709EF068802169588822AA58401A504321
:106A140003F010FF00252A467B4B03F06BFD03F0C7
:106A240067FE63218900744B585076490C60739952
:106A3400791A764A1160091A739175480160042025
:106A4400305E7E21595E1F46401A03F0F3FE044671
:106A54000E469020385803F0EDFE2246334605F0EA
:106A6400D3F92A46684B03F045FD03F041FE7399C0
:106A7400081A03F0DFFE2A46664B05F0C5F92A46DC
:106A8400654B05F0C1F95D9AD3052A4605F0BCF9BA
:106A940004460E466148046041609420385803F06F
:106AA400C9FE2A465E4B03F025FD2246334605F017
:106AB400ABF90246739071915A4802604160062016
:106AC4007099085E9821795E401A03F0B3FE04467B
:106AD4000E46A420385803F0ADFE2A46524B03F06C
:106AE40009FD2246334605F08FF92A464F4B03F041
:106AF400B9FB739A719B05F087F904460E467395AA
:106B040000224B4B03F0B4FD002811D10022204693
:106B14003146484B03F0CCFD002809D10022204621
:106B24003146394B05F070F903F0E2FD324A03E0D7
:106B340019200001304A1058E4215050729800285E
:106B4400709D0BD0E869296A884201DDE8692862F2
:106B5400E869696A884201DAE869686201213648AD
:106B64006891016035480068296E081ACD214900F2
:106B74005052334E301D7C22314604F0B1FF314F68
:106B8400381D39467C2204F0ABFFE8696790306019
:106B940028695390386059980546739E37463346A2
:106BA40007E0361D802E0D46719A1746729B2046CB
:106BB4004AD0244973968959CC176140091BB942BC
:106BC4000C4600DC3C467194A94200DB29461C4A71
:106BD4009259D4176240141B9C42224600DC1A4688
:106BE40072928442DDDB0446DBE7C046EC1200000F
:106BF400BC0E00201800005028000020FFFFFFFEFC
:106C04007C0F0020800F002000408F402C0F0020BC
:106C1400300F00200000084000005940900500207B
:106C240080842E418805002065CDCD410000F03FD1
:106C340000307140003071C0040F0020680F002044
:106C4400A00C0020A00B0020501AC1174840401A85
:106C54005190192801D300206890181BC11748408F
:106C6400441A074FF86D6821795A03F0B9FE1421CC
:106C740003F08EFE509484426F98024D05DB03E0CE
:106C84002800002001A000006898002800D0B8E285
:106C9400074842688368981AC1174840401A6799A0
:106CA4002492511ACA175140891A884203DC01E020
:106CB400A00C002008460449CC68E11ACA175140C8
:106CC400891A814203DC01E0A00C0020014604483B
:106CD4000569281BC2175040801A884203DC01E072
:106CE400A00C0020084604494E69711BCA17514084
:106CF400891A814203DC01E0A00C0020014604480B
:106D04008769B81BC2175040801A884203DC01E02F
:106D1400A00C002008460549C9694F91C91BCA1730
:106D24005140891A814204DC02E0C046A00C0020D4
:106D340001460548026A4F984E92101AC2175040F5
:106D4400801A884203DC01E0A00C002008460549B3
:106D54004A6A4E994D92511ACA175140891A814272
:106D640003DC01E0A00C002001460548826A4D982E
:106D74004C92101AC2175040801A884203DC01E07A
:106D8400A00C002008460549CA6A4C994992511A38
:106D9400CA175140891A814203DC01E0A00C00208B
:106DA40001460548026B49984892101AC217504090
:106DB400801A884203DC01E0A00C00200846054943
:106DC4004A6B48994792511ACA175140891A81420D
:106DD40003DC01E0A00C002001460548826B4798C3
:106DE4004692101AC2175040801A884203DC01E010
:106DF400A00C002008460549CA6B46994592511AD1
:106E0400CA175140891A814203DC01E0A00C00201A
:106E140001460548026C45984492101AC217504026
:106E2400801A884203DC01E0A00C0020084654903C
:106E34000548426C4498101AC1174840411A5498A6
:106E44008142269103DC01E0A00C0020014655910B
:106E54000548806C4390801AC1174840411A5598E0
:106E64008142289103DC01E0A00C002001465691E8
:106E74000648C16C43984291081AC1174840411A08
:106E840056988142299104DC02E0C046A00C0020FF
:106E9400014657910648016D42984191081AC1175D
:106EA4004840411A579881422A9104DC02E0C046C6
:106EB400A00C002001465C910648416D4198409128
:106EC400081AC1174840411A5C9881422B9104DC8E
:106ED40002E0C046A00C0020014661910648816D85
:106EE40040983F91081AC1174840411A619881425D
:106EF4002C9104DC02E0C046A00C002001466691FF
:106F04000648C16D3F983E91081AC1174840411A7E
:106F1400669881422E9104DC02E0C046A00C002059
:106F2400014620976891FA48016E3E983D91081AEF
:106F3400C1174840411A689881422F9100DC0146EC
:106F44002F467191F248416E3D983C91081AC11741
:106F54004840411A71988142309100DC014625462F
:106F64007291EB48816E3C983B91081AC1174840D6
:106F7400411A72988142319100DC014673911F924B
:106F84002196E348C26E3B98101AC1174840441A30
:106F940073988442329400DC04462593DC48036FE2
:106FA4001E92991ACA1751408E1AA642314600DC25
:106FB400214633942395446F1D93E21AD3175A4004
:106FC400D31A8B421A4600DC0A462297856F1C941A
:106FD4002C1BE7177C40E41B9442274600DC174631
:106FE400C06F1B951A90401BC5176840401BB842E0
:106FF400C84D00D905E1944200D902E18B4200D981
:10700400FFE03398864200D9FBE0739832998142BD
:1070140000D9F6E072983199814200D9F1E0719873
:107024003099814200D9ECE068982F99814200D9C7
:10703400E7E066982E99814200D9E2E061982C99A4
:10704400814200D9DDE05C982B99814200D9D8E0D7
:1070540057982A99814200D9D3E0569829998142B8
:1070640000D9CEE055982899814200D9C9E05498B6
:107074002699814200D8C4E0519803F0DBFB044612
:107084000D46509803F0D6FB02460B46204629468F
:1070940003F030FA0022A04B04F0B6FE03F028FB04
:1070A40015999E4B58522520C000185871903720CE
:1070B400C00073901A186798D0671698C000729031
:1070C4001B185398D8672498906795490D1DE0CDF7
:1070D40008694C6961948C696694CC6967940C6AFC
:1070E40068949D67259D55675E67239D15671F6797
:1070F400229DD566D86621989066619898668948DD
:10710400719C046020985066669858664F98106683
:10711400679818664E98D0656898D8654D989065BC
:10712400486A8C6ACD6A0E6B4F6B66978F6B679754
:10713400CF6B68970F6C719798654C9850655C6538
:10714400499810651D654898D064DE64479890643A
:107154006698986446985064679858644598106493
:10716400689818644498D063DF631F989063486CF0
:107174008C6CCD6C0E6D4F6D66978F6D6797CF6D70
:1071840068970F6E71979863439850635C63429855
:1071940010631D634198D062DE62409890626698E5
:1071A40098623F985062679858623E981062689857
:1071B40018623D98D061DF613C989061486E8C6E96
:1071C400CD6E0E6F4F6F67978F6F6897C96F719110
:1071D40098613B9850615C611E9810611D611D9817
:1071E400D060DE604B4D1C989060679898601B9847
:1071F40050605F60494F1A987399785072987199EA
:1072040039500020FE490860FE4E3768FE48006889
:10721400016840686A983C1A601E84416D98002891
:10722400589800DC002072905B9801406998814274
:107234003A4A01D100F0C7FC579161942520C1005E
:107244005058401C5C9150505F98002816D1F14B67
:10725400181F006801044B9A1040189C214008181C
:1072640050401860F84C6069F849491C0204629B5C
:1072740018400A401018294A5840A061D06D010CEA
:107284006B9B1C0C22464A439BB2594380B26793C2
:107294004343689460430C0C090459185441030C8B
:1072A4000004401869906341E94903C9014309D1C5
:1072B40000204B218900194A5158E64A5143E44AB7
:1072C4001160506066937197E34903C9014309D182
:1072D400002013210901114A5158DE4A5143DE4A64
:1072E40011605060E4260D4FB85900281CD4522078
:1072F400385A03F0EBFA0022D84B03F0FBF80446AB
:107304000D46B85903F096FA22462B463DE0C04696
:10731400A00C002001A0000000408F4028000020A5
:10732400A00B0020680F0020F86D6821795A03F043
:1073340057FB0446B85961428842B85929DA03F028
:1073440079FA73900D466A91204603F073FA024667
:107354000B460120C1076940739803F0CBF856909F
:107364000D465020385A03F0B1FA0022BB4B03F00B
:10737400C1F80022BA4B02F075FF02460B4656983C
:10738400294602F011FE739A6A9B04F03DFD03F056
:10739400AFF96A96709A906270205190385E916A43
:1073A400081A9062D169D06900290FD4C117AA4E76
:1073B4003268141875684D41002320462946A54AB1
:1073C40003F04AFB13210901785018E04042C11729
:1073D4009F4E3268141875684D4100232046294693
:1073E4009C4A03F039FB4B218900785078586C99FA
:1073F4004843F96D03F0F4FA4F2189007852346060
:107404007560709CA06A616BC217236B18182063A7
:107414004A416263A06AE16FC217A36F1818A0679C
:107424004A41E267A06FE16F00256B9A2B4603F097
:10743400FBFA2D21C90054917850606B216B699A35
:10744400511A669E3146814104DAF8203A50384692
:10745400F830466036988001391849683858401E1B
:10746400A9416A9C04DB052080013D503818456021
:10747400F96D3498385AD8227392BA5858235593D0
:10748400FB5A9A4210DD484303F020FA2A46734B14
:1074940003F030F803F046F93A59D317101A8B4128
:1074A40002DA70480088451C6E4805805620385A18
:1074B40029B2814228DD709C6663699820630020AC
:1074C400E067A067396E0A0C689E33465343679D94
:1074D4006A4389B24D437143160C1204AA185E41E3
:1074E4000B0C09048918734117221201B950B918F9
:1074F4004B6064997850639948605B2189007850A7
:107504006F99594A1170A065709E306B716B00259C
:107514006B9A2B4603F088FAF06230693A99C901F4
:107524006691795A88425EDA739838586C99884221
:1075340059DD4E490888401C088080B20A2854D37B
:1075440049480078002850D00A20088009204001CA
:107554003958474A914242D93858464988423ED818
:10756400549978580028785800D5404270645B20BC
:10757400800039583858002900D540423E49B0644B
:10758400706C0028084623D4432080003958F86DD5
:1075940081426C981CD2F86D0028374818D05D9849
:1075A400C0000A0C060C3746574383B25A4388B2CC
:1075B40043437043160C11045A187E412F4F010C9B
:1075C400000480187141709EFA6D002303F044FAA0
:1075D40005997852002024490870FBF7FFFF4920E1
:1075E40080003D5001E02148058064205690385ABF
:1075F400042800D9D8E005A1085C40008744C046AF
:10760400040F002024000020900E00200C784D71FF
:107614004000C04618000050F86D0023010C689D1E
:107624002A464A43679C614380B2444368430E0C34
:10763400090461185641040C000445187441F820EB
:1076440038583946F83142E000040050FFFFFF008B
:10765400A805002080EE3600B00500200000594047
:107664000000F0BF920F0020880F00208E0F002032
:107674000F0E000080FC0A00FFFF0000280000201D
:1076840011200201B858002838DD43208000385802
:10769400549979580818C11735E0386E002800D17C
:1076A40082E00023010C689D2A464A43679C61439B
:1076B40080B2444368430E0C090461185641040C1B
:1076C4000004451874411720010178587918496855
:1076D400F44A03F045F92A46234603F0A5F9054682
:1076E40062E05B2080003958002932D4002032E067
:1076F40054997858002835D4002035E0F86D549911
:107704007958081800213369669C3C5BB56C012DDF
:1077140002DBBD58EA1701E03D6E002269921A1996
:10772400D30FD3185A10DB1703F01AF900236C9AFD
:1077340003F07AF9DB4E3246002303F011F92A46AE
:10774400699B03F071F90546C0178543B5422ADAEF
:107754002AE038584042112109017A58002A08DCED
:107764003C6E0AE078584042432189007A58002A46
:1077740002DD7C58E11701E0FC6D00216991C1171D
:107784000026C84D2A46334603F0EAF82246699B90
:1077940003F04AF96A1E3346B341121A8B4100DBE7
:1077A4002E1A002900D4354601204E9000023D5087
:1077B400BD48026841681046084308D10021179863
:1077C40080003A58B9484243B748026041604C923D
:1077D400B74804684368204618436A9A08D10023CE
:1077E4002720C0003C58B1484443B148046043607A
:1077F4004D91B858002850934F940ED47220395AA2
:10780400B8584843642103F0C3F85F2189007850D5
:107814005198385E7958081A01E0F02038585F21F1
:10782400890078507A58D31773983858C11703F0E1
:1078340097F800236C9A549303F0F6F81722140176
:1078440053943D1969953A6E6B683E5986193E51B9
:107854004B416B60639C6368649D7E59301878511A
:107864004B416360100C689B19464143679C60431D
:1078740092B254435A43030C000426184B41100C93
:10788400110489195841699A5268539B1E46FB5842
:10789400CB1A0346934102DAB95169994860639B54
:1078A40058682A467959491E5499884101DBB950D0
:1078B4005960B858596800256B9C22462B4603F042
:1078C400B3F85B2189007850B85969994968224610
:1078D4006995002303F0A8F82F21C9007850379840
:1078E400C0003958385800290FD4C1174F9A1418BA
:1078F400509D4D410023204629466C4A03F0ACF8C4
:107904002721C90078506A4817E04042C1174C9AB1
:1079140014184D9D4D41002320462946634A03F027
:107924009BF87099C866486E6C994843F96D03F0EA
:1079340057F84F21890078525B48046045607424ED
:10794400385B0028B34900D19AE1385B0128084626
:1079540002D0385B0846103027990160385BAE4985
:1079640008807624385B002800D1A3E1385B012825
:10797400A849084602D0385B084610306299016075
:10798400385BA64908805C983858A54903F028F864
:10799400A4490968884204D0A24908600020FBF782
:1079A4001DFE5599785A7E5ACF2149009E4D2C6868
:1079B4007C5202F08BFF9D4A9D4B04F025FA02F0A5
:1079C40097FE73997F58874202DD002028600EE0FD
:1079D400304602F07BFF974A974B04F015FA02F009
:1079E40087FE874200DBF4E100208F490860934959
:1079F400086093490A46934F709E672080003A526C
:107A04004F208000385A0028084613D0F06E02F048
:107A14005DFF04460D46306F02F058FF02460B46E8
:107A24002046294602F066FD0022874B04F0ECF95B
:107A340002F05EFE8B21490078528448006A844932
:107A44004843000C83490968401A1649484382494F
:107A5400096802F09DFF814940180A2102F098FF4D
:107A6400CC22B8525A21785A669BF852B85E6A24DE
:107A74003B5F984238DAB85ABB5E6C22BD5EAB42BB
:107A840000DCB85ABA5E6E23FB5E3D5F95422C461D
:107A940010DC1446AA420FDA7D5E944210D1002015
:107AA40020E0C046A08601009805002080EE360044
:107AB400A0050020AA42EFDB2A467D5E9442EED068
:107AC400AB421E4600DB2E469D4200DC1D46A11A39
:107AD4000B467343AC1B00B2801A6043C01802F01B
:107AE40057FF709E669978525848C0695849484370
:107AF400C117090C401800145699414358480818F6
:107B04000A2102F045FFF0800620315E359AB25E0C
:107B1400305E914202DDD021785205E0D221795EB7
:107B2400884201DAF0887081484840695A9EB95BFE
:107B3400020C0B0C1C46544389B24A4380B24143A5
:107B44005843130C12048A186341010C0004801872
:107B540059410B227392002302F002FF02F0C4FE8B
:107B64000022404B02F0C6FC02F0C2FD15210901BF
:107B7400785236488069B95B020C0B0C1C4654439E
:107B840089B24A4380B241435843130C12048A1801
:107B94006341010C000480185941739A002302F0D8
:107BA400DFFE02F0A1FE00222E4B02F0A3FC02F045
:107BB4009FFDA92149007852579869902A4E3A4668
:107BC4002A4D719F619C2A486599405C518B00291C
:107BD40001D100F08DFC002801D000F089FC508B0D
:107BE4002449884200DDE5E0401E0A2800D9E5E288
:107BF4004000C046784480884000874448023D00E5
:107C04002E022B02DF02A3081B0237020B021C0107
:107C14009101C046180000508A0F0020860F0020F2
:107C240080510100380F0020440F00207B14AE4720
:107C3400E17AF03F0AD7A3703D0AEF3F3C0F0020E2
:107C4400FFFF00002800002000005940E00E002043
:107C5400E40C0000280F0020240F002030750000E1
:107C6400A015FFFF000024412400002001A0000013
:107C7400B8050020F1030000FAF79CFD00F035FC84
:107C8400F84800880028F84902D08320400039527F
:107C940083204600B85B002803D0B85B884200D03C
:107CA400EBE273983858B98E884200DBB7E00127BD
:107CB400FC48DAE2FC4800880028F94902D0412057
:107CC4008000395241208600B85B002802D0B85B9E
:107CD400884239D173983858398F8842F3482CDC5C
:107CE4006A9838583E21795E6C9A51438842F0482C
:107CF4000F994E9121DCCE21785E5E9ABA5E904255
:107D0400EC483A9A4E9218DCCC22B85E5E9BFB5E3D
:107D14009842E948529B4E930FDC785E6E99795EE7
:107D24008842E64836994E9107DBB85E6E99795ED3
:107D3400884209DA06204E90E14801F0F3FD4E989E
:107D4400B8536298DF490861B85B002800D117E690
:107D540073983858798F884200DB11E66A9838584E
:107D64003E21795E6C9A5143884200DB08E6CE20BE
:107D7400395E4222BB5E994200DB01E6CC217B5E88
:107D8400BA5E934200DBFBE53A5E46203B5E9A42D4
:107D940000DCF5E5795E385E814200DCF0E5B85B35
:107DA400022800D1ECE5C84801F0BCFD0020B8531E
:107DB400C448E3E5C549884224DCC549884200D16A
:107DC40069E1C249884200D0F8E16F9801F05EF899
:107DD4008BE3C04800680028BF4A02D1BD48076051
:107DE400384601460A318F42709E03DC0A388742C6
:107DF40000DBE5E100201060B6490860109AB74F37
:107E0400A749FAE5FD218900884200D1A0E1B449DF
:107E1400884200D0D2E10120FBF7E0FB65E36A98D9
:107E240038581299795E6C9A5143884200DBD5E147
:107E34000227AC4819E26194AB4802F09DFEA749C1
:107E44009C240859002800D102E2085902F0F2FCEF
:107E540000252A467395A54B02F04CFBA44A1668EC
:107E64007197576832463B4602F044FB0022A14B0F
:107E740003F0CAFF02F03CFC94226A9297498850AE
:107E8400709AD08898236793C85290889A226892EF
:107E9400885299483246994E3B46904D719F02F064
:107EA4006BFE285902F0C6FC739C22468F4B02F0ED
:107EB40021FB024692480B4602F05EFE6798285E5C
:107EC400904D02F0B7FC22468F4B02F013FB0246A2
:107ED4008E480B4602F050FE68988049085E02F016
:107EE400A9FC2246884B02F005FB024688480B4653
:107EF40002F042FE6A987949085802F09BFC224637
:107F04007C4B03F081FF024682480B4602F034FEAC
:107F1400814802F031FE2046FBF760FB619CE4E2FD
:107F24007E48164602F028FE6194CE24305BA021E0
:107F34007052705E02F07EFC0022734B02F0DAFA9B
:107F4400024677480B4602F017FE305F9821715EB7
:107F5400401A02F06FFC73906A9100226A4B02F09F
:107F6400C9FA02466F480B4602F006FE6E48719746
:107F7400076846686D483A46334602F0FDFD9C2486
:107F84005648005902F056FC0022584B02F0B2FA4F
:107F9400024667480B4602F0EFFD5048005902F0D4
:107FA40049FC0022514B02F0A5FA3A46719F334630
:107FB400524E02F09FFA00225E4B02F053F9739A7C
:107FC4006A9B02F097FA00225B4C234603F01CFFE5
:107FD40002F08EFBA421414A5050505802F02AFC72
:107FE40000222346619C02F085FA0022464B03F0EE
:107FF4000BFF0022514B02F035F9024650480B4664
:1080040002F0BAFD4F4802F0B7FD00203D4DFBF7EA
:10801400E5FA6AE2CC20105A8C215052505E7E213F
:10802400515E411A484800686C9A504302F0B0FC13
:1080340090212AE03120C000105890671346709AAE
:10804400D0880A99585290887E215852D06880214D
:1080540058501CE0FAF750FD47E20120FAF710FFF0
:1080640043E2C0468A0F0020FFFF0000D4201058CE
:1080740084215050505880215158411A3348006887
:108084006C9A504302F084FC8821144A505000201A
:10809400FBF7A4FA29E2002000F0F8FE25E2C0462E
:1080A400FFFF00009FC80008860F0020D8CA000800
:1080B400C0CA000894C60008E1C80008FDC400084E
:1080C400C0C8000818000050B6C60008F30300003A
:1080D400F20300003C0F0020440F00202800002081
:1080E400D2040000A8CA0008A2C5000800408F40BE
:1080F4009005002080842E411BC700082400002026
:1081040022C3000801A000000000594031C3000848
:10811400B4C50008B4C90008BEC500083CC30008C3
:1081240053C30008D4C500088805002062C30008B2
:10813400E2C500080000F0BF65CDCD410000F03F6E
:1081440095C30008C8C90008300F00202C0F002078
:10815400FC4B196A186A1A691A6900227592BB22C3
:10816400789206227492052212067A920D9A1206C9
:1081740079923F220A40194676928002800E7790C7
:108184005868002809D508460838F54A0260F54AB7
:1081940002604868002800D5AEE04868119908429A
:1081A40000D1B2E0ED49081FEF4A0260EF4A0260D5
:1081B40048681199084200D0A7E0A9E0EC4892E190
:1081C400EC4F6A9838585199795E88420FDA00204A
:1081D4001060E9490860E9498A1E0EE4CE20395E40
:1081E4004822BB5E99422BDD0327E5483DE0601C35
:1081F4001060E449884206D36A9838585199795AEC
:10820400401A089978520898385E0128DE4C13DB2E
:108214005C983858DD4902F0E3FB216888420BD0B2
:108224000899795EDA4D2A689309D21A51188A0995
:10823400029BFA5220602960D049699AFFF7DDFB5E
:10824400CC217B5EBA5E934207DD0427D1480CE063
:10825400D14801F067FB619C47E13A5E4C203B5EEC
:108264009A4200DB7AE30527CC4801F05BFBC14866
:1082740087530746CA4827990161B85B002801D192
:10828400FFF76CFB73983858F98E884201DCFFF7CE
:1082940065FB6A9838581299795E6C9A5143884202
:1082A40001DCFFF75BFBCE20395E4A22BB5E9942BC
:1082B40001DBFFF753FBCC217B5EBA5E934201DB0B
:1082C400FFF74CFB3A5E4E203B5E9A4201DCFFF71F
:1082D40045FB795E385E814201DCFFF73FFBB85B0A
:1082E400022801D1FFF73AFBAE4801F01BFB002046
:1082F400B853AB48FFF730FBAB4801F013FB974989
:1083040048681199084200D04CE7A84801F00AFBDC
:10831400A74801F007FB74A8F8F72AFC002864D0EA
:10832400A44801F0FFFA30688C490968609A114248
:1083340023D03168091A6C9A914226D28749096878
:10834400609A114219D03168091A6C9A91421CD270
:1083540082490968609A11420FD03168091A6C9AEF
:10836400914212D27D490968609A114205D0316860
:10837400091A6C9A9142D7D307E078490B688E4A60
:10838400521C0A608C490B4206D074494868119A01
:10839400104348604868A8E070490968139A11427C
:1083A400F3D03168091A6C9A9142EED26B4909688C
:1083B400139A1142E9D03168091A6C9A9142E4D2B5
:1083C40066490968139A1142DFD03168091A6C9A18
:1083D4009142DAD261490968139A1142D5D03168C1
:1083E400091A6C9A9142D7D3CFE730685B49096880
:1083F400609A114223D03168091A6C9A914227D2AB
:1084040056490968609A114219D03168091A6C9A60
:1084140091421DD251490968609A11420FD03168C6
:10842400091A6C9A914213D24C490968609A114214
:1084340005D03168091A6C9A9142D7D308E04749AC
:108444000B685D4A521C0A605B490B4200D1E1E1B2
:108454006194424C606811990843606060685748B1
:1084640001F060FA30682168619C609A114227D05B
:108474003168091A6C9A91422BD238490968609A7A
:1084840011421DD03168091A6C9A914221D23349A4
:108494000968609A114213D03168091A6C9A9142A2
:1084A40017D22E490968609A114209D03168091A15
:1084B4006C9A91420DD229490968609A1142D7D128
:1084C400264B19683C4C621C1A602142619C00D105
:1084D400D0E122494868079A104348604868384800
:1084E40001F020FA374801F01DFA002021494883A1
:1084F400729820406D9A121A334800685E990840B9
:108504006D92104322D130683168091A0A290BD8B8
:108514003168091A0A2907D83168091A0A2903D8BF
:108524003168091A0B29EFD32748006840060BD499
:108534006298F4306D905F980028244E48D0002053
:108544004AE0C0461020024000206D901F4E307D4E
:108554000028394647D1FDF784FDC046102002406B
:1085640023016745AB89EFCD3B2A19087F6E5D4C2B
:1085740014CA0008280000203C0F0020FFFF000060
:1085840064C60008312A0000400F00208051010019
:10859400480F00207EC8000838C70008DAC4000865
:1085A4001800005086C60008C7C4000840C600086A
:1085B40060CA000869C80008FA83000070CA00088D
:1085C40056C6000888CA000810080050B8050020E4
:1085D4004B98F749086001205F90307D00283946A8
:1085E40001D1FDF73EFD4A98C0007390315805292A
:1085F40001D2FDF72DFD71972723F05C72900120C5
:1086040037466A90C6438C1E26402837F74A02E054
:10861400BF1CB61E73D0781E007850404208C007B5
:108624001AD06A405008D20719D14208C0071AD09C
:108634006A405008D20719D14208C0071AD06A40CC
:108644005008D20719D14508C0071AD0E848454058
:108654006A08E80718D119E05008D207E5D0684045
:108664004208C007E4D15008D207E5D06840420868
:10867400C007E4D15008D207E5D068404508C007D8
:10868400E4D16A08E80701D0D94842403D78554012
:108694006808EA0705D0D64D68404208C00704D1EF
:1086A40004E0D34D4208C00700D06A405008D20706
:1086B40012D068404208C00711D15008D20712D026
:1086C40068404208C00711D15008D20712D0684050
:1086D4004208C0079CD010E04208C007EDD06A40B1
:1086E4005008D207ECD14208C007EDD06A405008C8
:1086F400D207ECD14208C0078AD06A4088E7C8078D
:1087040005D1BC4E719F481C2CD1FDF7A1FC084635
:108714006A9DA843B74E30182525405D424090B26B
:108724004008B34DD20757D06840719F4208C00734
:1087340056D15008D20757D068404208C00756D1D6
:108744005008D20757D068404208C00756D1500895
:10875400D20757D068404208C00756D1481C01D1FF
:10876400FDF776FC3019C05C7118659BC95C090281
:108774000818904201D0FDF76BFC7298002806D0CF
:108784009D48008B7299884201D0FDF761FC5F9887
:108794000028394601D0FDF764FC0E992831729BFC
:1087A40073548B208500002474510B98325C102A7A
:1087B400689500D1A2E0062A00D18BE0032A00D0FC
:1087C400A6E08D48008B002B00D1B8E0984200D180
:1087D400B5E00B228623FDE0719F4208C007A8D0B4
:1087E4006A405008D207A7D14208C007A8D06A40FF
:1087F4005008D207A7D14208C007A8D06A40500841
:10880400D207A7D14208C007A8D06A40481CA9D102
:10881400FDF71EFC79490968139A114200D117E645
:108824003168091A6C9A914200D311E673490968B8
:10883400139A114200D10BE63168091A6C9A9142DD
:1088440000D305E66D490968139A114200D1FFE58A
:108854003168091A6C9A914200D3F9E567490968AD
:10886400139A114200D1F3E53168091A6C9A9142C6
:10887400D0D3EDE561490968139A114200D128E685
:108884003168091A6C9A914200D322E65B4909685F
:10889400139A114200D11CE63168091A6C9A91426C
:1088A40000D316E655490968139A114200D110E61F
:1088B4003168091A6C9A914200D30AE64F49096853
:1088C400139A114200D104E63168091A6C9A914254
:1088D400D0D3FEE54848008B002B01D0984213D139
:1088E40034462734E378A2781002C018629DDB3541
:1088F400A8423AD92520C000414A57E03E48008B9F
:10890400002B0CD098420AD02520C0003D4A4DE0EF
:1089140070186A9B8370099B5A4042705DE032462E
:108924002732577910790002C31918467C387B2402
:10893400E443A0422AD82520C000392235E032463B
:108944002732567910790002801905467E3D0A9B2C
:10895400DF438323BD422DD203223AE0795E385EA1
:10896400814200DB89E4062770E44000224F3D1871
:1089740026796E7064793C541E484018447106711F
:108984001C4EC37082700624447027E07297D57819
:108994009478200242199F181B4BD819401E984204
:1089A40000D352E12520C000069A1201325214E08D
:1089B40018000050D57897783A02729552198518A4
:1089C400669511484019401E0F4DA84200D37AE124
:1089D4000222084E701882704370032425466A9858
:1089E400854372182E46014F14E0C046FFFF000075
:1089F40001A00000B805002028000020102002403B
:108A040086020000860B000024FEFFFF921CB61EA7
:108A140000D181E013787B405808DB071DD0DA4B86
:108A240058404308C0071BD15808DB071DD0D64B5C
:108A340058404308C0071BD15808DB071DD0D24B50
:108A440058404308C0071BD15808DB071DD0CE4B44
:108A540058404308C0071BD11CE04308C007E3D0BB
:108A6400C94843405808DB07E1D14308C007E3D0B5
:108A7400C54843405808DB07E1D14308C007E3D0A9
:108A8400C14843405808DB07E1D14308C00701D07F
:108A9400F848434057785F407808FB071DD0F54BF2
:108AA40058404308C0071BD15808DB071DD0F14BC1
:108AB40058404308C0071BD15808DB071DD0ED4BB5
:108AC40058404308C0071BD15808DB071DD0E94BA9
:108AD40058404708C00799D01BE04308C007E3D0BB
:108AE400E44843405808DB07E1D14308C007E3D01A
:108AF400E04843405808DB07E1D14308C007E3D00E
:108B0400DC4843405808DB07E1D14708C00700D1DF
:108B14007CE7D848474079E7E00703D13A0AD44BC9
:108B2400689D3DE0D24B5819405C4740B8B24008BC
:108B3400D04DFA0719D068404208C00718D1500830
:108B4400D20719D068404208C00718D15008D2078C
:108B540019D068404208C00718D15008D20719D06C
:108B640068404708C00718D118E04208C007E6D09B
:108B74006A405008D207E5D14208C007E6D06A40EF
:108B84005008D207E5D14208C007E6D06A40500831
:108B9400D207E5D14708C00700D06F40689D3A0A64
:108BA40018194754401842700C20659A9854A41C14
:108BB4005C51A2B2504250411A6813467C335D683E
:108BC400202D6F9D00D10546002D719F34D19668EC
:108BD4000C98864202D1106900282DD018780128FB
:108BE4002AD0104654304480DD600480A0484018E8
:108BF400106537985860506E019988420DD10C98D1
:108C0400864203D1106900289E4800D09E481D70FA
:108C140010671168083103980BE00C98864203D161
:108C240010690028954800D095481D701067116898
:108C340009980A6802430A6000208D49739A885093
:108C4400087539468B4DFDF70CFA619568006694FA
:108C540063021818854B1D180026AC198448831923
:108C64002E20185C60702F20185CA855501CB84248
:108C74001BD23020185CE0703120185CA070901C6E
:108C8400B84212D23220185C60710498185C2071CA
:108C9400D01CB84209D23420185CE0713520185C2D
:108CA400A0710836121DBA42D7D3714E7018729A49
:108CB400427100220271619AC270669A8270102217
:108CC400427006248AE66A4D681873002E46837043
:108CD40003234370729840007B021818634B1818E2
:108CE4007290669D6791301972990B195F78952679
:108CF400760087558719085D7870501CA84219D2F0
:108D0400D878B8709878F870901CA84214D2587922
:108D1400387118797871D01CA842554E67990FD2D2
:108D2400D879B8719879F8710834121DAA42DAD347
:108D3400E41C53E6641D00E0E41D4D4E67994DE6C6
:108D440009344BE6BFF34F8F444914394A4808604D
:108D5400BFF34F8F00BFFDE730682168C90701D01A
:108D6400FDF786F8A168C90705D1A1683D4A1140FD
:108D7400589A1143A1603168091A0329EDD3216877
:108D8400C907EAD1FDF737F801A000000A68A56811
:108D9400344B1D40034658980543A560579802403C
:108DA4009A18D2082369119DAB4229D25B98830497
:108DB4002D4D2D681D40AB0C072B21D3DB1E589D78
:108DC4009D407B957B9B5B087B937B9B002B17D003
:108DD4007B9B5B1E7B937B9B002B11D07B9B5B1E41
:108DE4007B937B9B002B0BD07B9B5B1E7B937B9BA2
:108DF400002B05D07B9B5B1E7B937B9B002BE7D1D9
:108E04000B685798834313430B60A168154A1140BC
:108E14000F9A1143A1603168A268D20712D0326858
:108E2400521A032AF8D3A268D207F5D00C4A906DDF
:108E3400102101439165D06D58990843D065D05DE8
:108E4400FCF7B1FFE16872980143E1600448806D6A
:108E5400589908430F998843FCF706FE20ED00E07B
:108E6400840D0020E8FFFF7F082701402800002030
:108E7400B805002001A000000400FA05B1130008A1
:0C8E84005FC1000855130008FFBC000887
:108E9000F0B589B00021069103910291F14C216A4D
:108EA0003F220A400492216A8902890E05912569B0
:108EB000ED49079122690A40089200284DD0EB48FD
:108EC00000F032FDE8B2AA2800D08DE0BB20069069
:108ED00002200290606800280BD520460838F84927
:108EE0000160F84901606068002802D5F64800F08A
:108EF0001BFD0126B5076068400007D5201FF44917
:108F00000160F44901606068284202D0FA4800F02C
:108F10000BFD0195FA4800F007FD02A8F7F72AFEBD
:108F20003704002864D0F74800F0FEFCEB480168E5
:108F300022683A4200D0B1E02268E94B5D1C25600E
:108F40001A4203D12268520300D5E5E06068019916
:108F500008436060606809B0F0BDE8B2AA2800D19B
:108F6000D6E0CC2800D1D3E0AA20069002200290BF
:108F70006068002809D520460838D1490160D149E8
:108F800001606068002800D5C4E0D04800F0CCFC47
:108F9000606840002AD50126B507201FCC49016032
:108FA000CC4901606068284220D1CB4800F0BCFC6D
:108FB00002A8F7F7DFFD002800D1D4E0C748016818
:108FC0002268D20300D525E12268C54B5F1C2760CB
:108FD0001A4203D12268520300D549E16068284350
:108FE00060606068BF4891E0C4488FE0C2488DE08F
:108FF0000096BA4E7D2130682268CD003A42B84BC7
:109000002FD121685A1C2260194203D121684903DB
:1090100000D5B7E060680199084360606068B348B4
:1090200000F082FCAE4B3068216839425CD0316878
:10903000091AA94260D22168394255D03168091A0B
:10904000A94259D2216839424ED03168091AA94241
:1090500052D22168394247D03168091AA942E3D374
:109060004AE03168091AA942D4D221683942C8D0ED
:109070003168091AA942CDD221683942C1D031687C
:10908000091AA942C6D221683942BAD03168091AF0
:10909000A942BFD221683942E3D1B2E77D22D20092
:1090A00003685B1A934200D350E723683B4200D128
:1090B00042E703685B1A934200D347E723683B42C9
:1090C00000D139E703685B1A934200D33EE7236877
:1090D0003B4200D130E703685B1A934200D335E787
:1090E00023683B42DCD127E721685A1C22601942E1
:1090F00002D1216849036BD40098C007616801431D
:10910000616060687A4800F00FFC7F4800F00CFC5A
:1091100009B0F0BD6C48F9E7B2047D23DB000568B7
:109120006D1A9D4200D311E72568154200D10DE765
:1091300005686D1A9D4200D308E72568154200D1E5
:1091400004E705686D1A9D4200D3FFE625681542C5
:1091500000D1FBE605686D1A9D4200D3F6E625684E
:109160001542DCD1F2E6604800F0DEFBF7F7BCFB0D
:109170005E4800F0D9FBF7F759FB5D4800F0D4FBDF
:109180005C48C3E7009989043268121AAA4200D3E6
:1091900040E722680A4200D13CE73268121AAA422C
:1091A00000D337E722680A4200D133E73268121A47
:1091B000AA4200D32EE722680A4200D12AE7326889
:1091C000121AAA4200D325E722680A42DCD121E71D
:1091D000009989043268121AAA428DD222680A4282
:1091E0008AD03268121AAA4286D222680A4283D0F2
:1091F0003268121AAA4200D37EE722680A4200D1DE
:109200007AE73268121AAA4200D375E722680A4246
:10921000E0D171E732047D23DB0007687F1A9F42AB
:1092200000D3DBE62768174200D1CDE607687F1A36
:109230009F4200D3D2E62768174200D1C4E60768F0
:109240007F1A9F4200D3C9E62768174200D1BBE6C8
:1092500007687F1A9F4200D3C0E627681742DCD117
:10926000B2E6C0461020024000604F0740CA000826
:10927000B2047D23DB000668761A9E4200D3ADE679
:109280002668164200D1A9E60668761A9E4200D3E7
:10929000A4E62668164200D1A0E60668761A9E4229
:1092A00000D39BE62668164200D197E60668761A38
:1092B0009E4200D392E626681642DCD18EE6C04676
:1092C00023016745AB89EFCDC7C400082EC600084F
:1092D0003B2A19087F6E5D4CF5C70008240000206A
:1092E000FA8300002BC8000824CA000870CA0008CE
:1092F00056C600080AC8000840C600084CC8000846
:0C93000060CA000869C8000888CA00089C
:10930C0006480168002908D10168002905D10168C7
:10931C00002902D101680029F3D07047580F0020B2
:10932C000C490868401C08600B480268521C02601B
:10933C00D2087D2A0CD30968084A914208D30849FF
:10934C00CA6D521CCA6500220260886D401C88657B
:10935C007047C04624000020340F0020214E00002E
:04936C00F0000020ED
:10937000F0B583B03748001F0568374A1468206885
:1093800004260190304041424141106C1C230340AF
:1093900037469F40384602952840424242410A43A0
:1093A00030D0009401200226019D2A4632405142CD
:1093B00051419E40029A1642074600D00F46002FA8
:1093C00032D008210D4069426941DA40120700D5C8
:1093D0000846002826D1242000211F4C2154009A41
:1093E00010680E2188431060012001469940194BF6
:1093F0001A680A431A60E06325216054616B0029F2
:109400000ED10FE02068800602D42068B0432060AF
:1094100010490868384308600F48016B002901D0E3
:109420000D48884703B0F0BD2346206880060A4AED
:1094300006D418680A218843186025200121115498
:10944000242017540349086830430860D16A002972
:0C945000E6D1E7E704000240E80D002030
:10945C00F0B58AB098480168C8690A6809924A68E8
:10946C0001220792120706928A68089204074FD0CD
:10947C00069A531C089A134001252A0216462036D8
:10948C00099F3E401E4343D03A4056425641C207C4
:10949C00079A00D03246002A05D10D628822864FE9
:1094AC00BE582E43BE50089A15406A426A41860740
:1094BC00079E00D51646002E08D102220A62882289
:1094CC007D4EB658042737437B4EB7506A426A41EB
:1094DC004507079D04D4002D04D0002C0CD417E0B4
:1094EC001500FAD104220A628822734FBD58022655
:1094FC002E43BE50002C0BD52022099C2240134336
:10950C0006D008220A6288236B4DEC581443EC50A9
:10951C000125EA050492020513D5089A049B1A400A
:10952C00AB06099C23409A180BD0EA020A628422EB
:10953C002023614CA3508022A350604A1575604BC8
:10954C00D554202203460592134003931CD0089A4D
:10955C00069B1A40099B059C2340134314D04522BB
:10956C00D200564B9C588426534FBE59222E30D1D4
:10957C002E02B4422DD21C194E6A2727E655504CA8
:10958C001D559C58641C9C50802306461E403DD0A3
:10959C00089A049C2240099C1C40144336D0474A2C
:1095AC001268D458212C1DD1174656373C88002CF4
:1095BC00146802941FD0146D019424780097029FB4
:1095CC00BC62019C641C1465009C2288521E228083
:1095DC0018E08A69082313438B61802306461E40DA
:1095EC00D6D113E0126814689C43146014684027A9
:1095FC002743176006E022689A43226022684027BE
:10960C0017432760232212012C4CA55402954027A6
:10961C00099C3C4062426241400600D50792079883
:10962C0000280CD10868B8430860234D0598E85011
:10963C00244800220270842022242C502A6788227D
:10964C001D48805800282BD0842022241A4D0790C6
:10965C002C500398002809D0089D039106992940A5
:10966C00099D059805400D4303991BD1002E17D079
:10967C00089D049A1540099A1A402A4310D00A688A
:10968C00BA430A600C4D0598E85007982C502620D8
:10969C000A4900220A5423200001029B0B542A671A
:1096AC000AB0F0BD8869082303438B61002002498E
:1096BC0088500AB0F0BDC046940A0020B8050020BE
:0896CC0031020000DE05002060
:1096D40001204102074A13689B0503D453680B42D7
:1096E40004D17047116053680B42FAD051600249AB
:0C96F400086070470C180240040F0020B2
:10970000F0B583B05D4C2068C5680226294631401B
:109710004A424A410769394631404B424B41134363
:109720002346574A0ED11146FE31016101211977B6
:109730008069800704D05148F8F722F9504A23463F
:109740000020187701240420294601900140484256
:1097500048417907214600D50146032000020290C6
:10976000002910D118681146FC3101611E7780690B
:109770000299084205D041481E46F8F701F9404ACF
:109780003346002018770826294631404842484190
:109790003907214600D5014600290FD11868114626
:1097A000F831016101991977C069800704D0334805
:1097B000F8F7E6F8324A314B00201877102129409B
:1097C00048424841F906214600D50146002910D1FA
:1097D00018681146F03101611E77C069029908428C
:1097E00005D026481E46F8F7CBF8254A3346002018
:1097F00018770121294048424841F907214600D005
:109800000146002903D118681146FF31016180200B
:109810002840414241414122D2011742224600D014
:109820000A46002A02D11968164A0A61414241419A
:10983000F805204600D508460028114A01D11868CD
:10984000026140212940484248417906214600D51D
:109850000146002903D118681146C031016120205A
:10986000054068426841B90601D403B0F0BD040068
:10987000FBD11868E032026103B0F0BD440E002055
:08988000FFFEFFFF7FDFFFFF89
:10988800B0B51E4D2C1F20688006400F411E0329CD
:1098980022D81B487944097949008F442301171AB3
:1098A800296803220A40032A00D016482968490675
:1098B800490F491C01F092F829684904490E4843A8
:1098C8002968490F491C01F089F80BE07D20000246
:1098D80008E00120C00305E00C3D28688004410F22
:1098E8000848C84008490860226892093C23134088
:1098F800064AD258D0400860B0BDC0460C1002409D
:1099080000127A000024F4002000002090BB000818
:1099180080B50249096802F048FA80BD14000020A9
:10992800B0B5044608480568204602F04BF80246E0
:109938002846214602F079FB401C03D00A20FFF795
:0C994800E7FFB0BDC043B0BD140000201C
:10995400C20F490089184000034A40428A4101D39A
:0C99640000207047012070470000E0FF69
:109970000122D2079143034A4A40104341424841E1
:089980007047C0460000F07FB3
:10998800074A0A40531E9A41C00F49000818054962
:10999800884201D3002000E0012010407047C046F3
:0899A8000000F07F0000E0FF69
:1099B00030B50E4B5D1C0C0D2C4010D0AC420ED0BF
:1099C000A2189A4205DD0120C00701400948091884
:1099D00009E0002A04DD064B19401205114330BD91
:1099E0000120C0070140002030BDC046FE07000036
:0899F000FFFF0F800000F07F73
:1099F80010B54B005B0D084CA34201D0002B02D1DF
:109A08000023136010BD054C1B191360044A114054
:109A1800044A891810BDC046FF07000002FCFFFF7A
:089A2800FFFF0F800000E03F8A
:109A3000F0B587B00E4604460021C843574F069044
:109A4000401C0590384601914841590004914D0D44
:109A5000534900D18CE0E50F71000291491903913F
:109A6000650006994D1B03998F4100D282E0D10F0A
:109A7000049D69185500059F7D1B88417AD30121FB
:109A8000C807304004904748354605400340101B46
:109A90001846A84171D2039109050298470D059116
:109AA00003D0481E06400E430DE08D420AD20398B3
:109AB000C004E10F6E00761864007F1E85423546B3
:109AC000F7D300E02E461D0D3748054004D0059918
:109AD000481E03400B430FE0059883420CD20398C5
:109AE000C00406901946D30F4800C31852006D1EDB
:109AF000069881421946F6D3AF4212DDA01A3146CC
:109B0000994104D454405E40264302D113E02046DC
:109B10003146C40F49000E1944007F1EAF42EDDCF0
:109B20002F462046841A35469D41059906D450405B
:109B30005E40064304D1019C049916E00446354674
:109B40000D420AD10398C004E10F6A005118640065
:109B50007F1E05420D46F7D000E02946002F15DD97
:109B6000781E049A891800050918204607B0F0BD30
:109B7000019CFAE7019C0A49F7E762405D40154302
:109B800000D00496002DD7D10024D5E70398C21B3E
:109B9000204600F0C7FE04460020E2E7FFFFDFFF9B
:0C9BA0000000F87FFFFFFF7FFF070000C0
:109BAC00F0B583B00D46044628494A1C280D1040D8
:109BBC00421E8A4240D22749884205D20024002DF9
:109BCC00264635DA264E33E03331884201D92E460B
:109BDC002EE01F49461820462946324600F08CFEDE
:109BEC001D4A114001434A424A410020002D01DA2E
:109BFC00014600E0012111430291184901903246BF
:109C0C0000F09AFE074632460E462E402740019B36
:109C1C00D843401C1049594100F07EFE029A381876
:109C2C007141002A00D10E46002A00D107463C465D
:109C3C002046314603B0F0BD002802D10121C907EE
:109C4C000D402E460028F3D10024F1E7FE0700005A
:109C5C0001FCFFFFFF030000FFFF0F000000F0FFFF
:049C6C000000F0BF45
:109C7000F0B587B00A0D521E484B9A4214D206AA7C
:109C8000FFF7BAFE06460F464948301A4748814159
:109C9000069C3046394618DA0022474B00F0E4FAB9
:109CA00006460F46641E14E0C30F4A00D318440052
:109CB00064423B4C9C416AD3520D6CD000290A4649
:109CC00000DA394A002963DA66E00022394B00F0F5
:109CD000CBFA059403900D460024E24304943046E9
:109CE0003946FFF765FE354B002200F0BDFA02460B
:109CF0000B460398294600F0FFFB03900F460246EF
:109D00000B4602F083F804460D462D4E02213046E4
:109D100022462B4602F085FA2A4A2B4B00F0A4FA81
:109D20000290019110360321304622462B4602F064
:109D3000A0FA02460B460298019900F0DDFB22468C
:109D40002B4602F063F8039C22463B4602F05EF885
:109D500022463B4600F088FA06460F46059800F07A
:109D60006BFD04460D46194A194B02F04FF8324676
:109D70003B4600F079FA06460F46164B2046294628
:109D8000049A02F043F832463B4600F06DFA0A4668
:109D9000114607B0F0BD034A0020F9E7FE070000B6
:109DA0000000E0FF0000F0FF0000F87F9EA0E63F0B
:109DB000CE3B7F660000F0BF0000E0BF0000E03F48
:109DC000C00000089AB5B312FF0750C0A80C615C30
:089DD00010D02BBF0030E63F6C
:109DD800F0B585B00C4607465948411C220D0A408B
:109DE800511E814200D38EE05948C01B5748A041FC
:109DF80000DAA2E000205849C91B5649A141014692
:109E08007FD30120C007214681435648381A544859
:109E1800814174D3544A554B3846214601F0F2FF2C
:109E28000122D2072240524BD31800252A46049516
:109E380000F016FA00F05AFC039000F0F9FC0290CA
:109E48000E464C4B002201F0DDFF3A46234600F057
:109E580007FA04460F46484A484B0298314601F033
:109E6800D1FF22463B4600F0FBF906460D46024666
:109E78000B4601F0C7FF0F46414A424B0446029089
:109E880001F0C0FF404A414B00F0EAF922463B4648
:109E980001F0B8FF3E4B049C224600F0E1F932463F
:109EA8002B4601F0AFFF05460E46204630492A46AC
:109EB800334600F0B9FA01900091364A364B029CBD
:109EC8002046394601F09EFF344A354B00F0C8F968
:109ED80022463B4601F096FF019A009B00F0C0F92C
:109EE80002460B462846314600F002FB049A204BF6
:109EF80000F0B6F9039A521CFFF756FD01E0174926
:109F0800002005B0F0BDF80F61000818790049423B
:109F18000C49814121460ED30120C00781430A48DC
:109F28004840384300D075E7002C214600DA00216C
:109F3800002C00DA00273846E3E70349E0E7C0468B
:109F4800FE0700000000E0FF0000F07F422E864080
:109F5800EF39FAFE2B2386C0D2BC7ADD0000F03F31
:109F6800A19CC73B2342920C3CF92F9E2C15F73F2E
:109F78000000E03F0030E6BFA80C615C10D02B3F2A
:109F88001CDC586FA452F13EE0F6B36FE4707C3FDE
:109F98000000D03F0938DE6F993F403FB35142710E
:049FA8008E71AC3FCB
:109FAC00F0B585B016460024E7438B4D7A1C2A4643
:109FBC0062414A4002436FD001955A00550D00D1C1
:109FCC0008E100940290874C601C039104930D0DE2
:109FDC0005406D1EA54273D21D461C0D0440824BDC
:109FEC00E4185B1C9C426BD337463046294600F084
:109FFC007BFB064600F01AFC2A46029D7840514035
:10A00C000143039C30D101200290C00786422BD023
:10A01C00002E0096714B41D0F0174640361A00279F
:10A02C0001970393012E019A00D02A460497012E22
:10A03C006A4B00D023462F462846214601F0E0FE0D
:10A04C00224605460C46304602990840634B00D028
:10A05C00134642423A400498039901F0D1FE074658
:10A06C000B467608DDD11AE000222846214613461D
:10A07C0000F01AFB002802D0604900241DE00120EA
:10A08C00C007844328462146FFF7ECFD3A46049B63
:10A09C0001F0B6FEFFF79AFE04460EE00027002002
:10A0AC004E493A461D4600F021FA04460098002815
:10A0BC0000D42946002800D43C46204605B0F0BD0B
:10A0CC000298C30F4C00E3184400641E484C5C41DA
:10A0DC00E2D20125F30FD21873005B1B434B9A415C
:10A0EC0010D23F4A114210D0424B0C465C40044304
:10A0FC0026D00C4654400443049827D100283CDA5F
:10A10C002146DAE734460499D7E737463046049CB3
:10A11C00214600F0E9FA064600F088FB4C403B462D
:10A12C004340234327D1049900291C46194600DAE1
:10A13C002B49F007C1D0E807039E06407118BCE715
:10A14C000094049800281ADA009819E05840064345
:10A15C0002982CD1284A4A400243009C1F49ACD09B
:10A16C00EA07039B93430022391A0198984114463D
:10A17C002ED31B4A2CE0049A3FE711469DE710466C
:10A18C0003903046049F394600F0AEFA044600F0C6
:10A19C004DFB794070400843039802D1E8070399BE
:10A1AC000818E10700D00390009C039985E7EB07A2
:10A1BC000C469C430023391A0198A0411C461946B1
:10A1CC0000D37AE70C48039E46400298304301D0F6
:10A1DC00114672E7014970E7FFFFEF3F0000F03FC7
:10A1EC000000F07FFE07000001F8FFFF0000E0FF19
:10A1FC00FFFF1F000000F0FF0000F0BF0000F87F21
:10A20C00F0B581B000280090124D13D00146C01754
:10A21C0041400F1A0026104CF80707D00CCC3046E2
:10A22C002946083C01F0ECFD06460D4608347F0833
:10A23C00F2D100E000260020064932462B4600F001
:10A24C0055F9009A002A00D43046002A00D4294639
:0CA25C0001B0F0BD0000F03FE800000879
:10A26800F0B40125ED070F005F405AD48B4200D1AE
:10A27800824205D950404240504059404B405940D5
:10A288004E18760DDF187F0D3BD0741C640529D05D
:10A29800F41B352C26D80E0DDB022B43DB0AC90232
:10A2A8002943C9121700202C1ED2E741E24057402B
:10A2B800E3415A40A340E3405A40002480185941E2
:10A2C8000AD3B21C520521D0C207012F62411700E0
:10A2D8004008CB0718434908013636054208AF4104
:10A2E80060417141F0BC7047203C06D01F00E74137
:10A2F800E3405F400024012A6741C0186141EBD365
:10A30800DFE7002EEED129400020EBE701363105CA
:10A318000020E7E7E742E5D10020C143090DC90461
:10A32800E0E76B400E00871A9E4104D26E40C01BC6
:10A33800B141D21973414E18DF18AC0AE642E9D28E
:10A34800760D7F0D31D0F41B362CCBD8B4460E0DCC
:10A35800DB022B43DB0AC9022943C90A012C32D884
:10A3680004D1D4075208DF073A435B08EF0A644276
:10A37800904199411ED0002239424DD124194041C3
:10A3880049410124394204D1013400184941394274
:10A39800FAD06246A24204D9361B013E3605891915
:10A3A800A0E7F10AC90700209CE736429AD10020AD
:10A3B800002197E70200224394D0B842DED2010080
:10A3C80020002024E3D1202C13DD203CE24117009B
:10A3D800A240E2405740E3415A40A340E3405A407C
:10A3E800012FBF410137174300227C429841914118
:10A3F8000CE01700E741E2405740E3415A40A340D0
:10A40800E3405A407C429041994100220F0303D215
:10A41800013E241940414941013E36054708AC41F7
:08A4280050417141F0BC704786
:10A43000F0B40125ED076B40004C20476FA20008E7
:10A4400030B405004D400124E407254042004B0094
:10A45000120E32D01B0E3CD0FF2A33D0FF2B3FD040
:10A46000D21800022043000A09022143090AC4B29B
:10A470004C43000AC3B24B43000A4843210A5B180D
:10A48000190A091801D44900013A080A7F3A2ADB5F
:10A49000FE2A0FD2D2051C43240601D001242143F9
:10A4A000C9B280295041802901D140084000284389
:10A4B00030BC7047FF20C005F9E71B0EFF2B0AD008
:10A4C0002800F5E7400206D1FF2BF3D1490202D163
:10A4D000F0E7FF2AF4D17F2000010C300005E7E708
:10A4E0004902F8D1E6E743020132E9D15B120233B7
:08A4F000E6D9D805E4E7C046F7
:10A4F800F0B40125ED070C005C402C40A446AE0AE0
:10A508004C18DF18F4423DD2F74245D2640D4CD0C6
:10A518007F0D3CD0E41BC9022943CF0ADB022B4341
:10A52800DB0A0600B61A9F4104D2013CB6197F41E6
:10A53800B6185F416812800D241838DD001884426F
:10A5480025D8E80C0021B6197F41B61A9F4103D3DC
:10A5580040414941F7D304E0B6185F41001849412A
:10A56800F1D32405B6197F41B61A9F4105D3374365
:10A57800C20717430022012F50416141624611432F
:10A58800F0BC70470CD100280AD1F74208D200204D
:10A59800C143490D0905F1E7002A01D1F74206D068
:10A5A8000020C143090DC904EAE77F0DF8D0002057
:04A5B8006146E5E72C
:10A5BC0030B401256D054C00E54215D85C00E54230
:10A5CC0012D80C001C436400044314430FD005D272
:10A5DC0082428B418041013030BC7047904299419E
:10A5EC008041013030BC7047002030BC70470120E6
:04A5FC0030BC7047B8
:10A6000070B4012676054C005D00E6420CD8EE429F
:10A610000AD825430543154303D0994204D19042FB
:10A6200002D1012070BC7047002070BC7047C0464A
:10A6300030B401256D054C00E54215D85C00E542BB
:10A6400012D80C001C436400044314430FD005D2FD
:10A65000904299418041013030BC704782428B4129
:10A660008041013030BC7047002030BC7047012071
:04A6700030BC704743
:10A6740030B401256D054C00E54215D85C00E54277
:10A6840012D80C001C436400044314430CD005D2BC
:10A6940082428B418041404230BC70479042994194
:10A6A4008041404230BC7047002030BC7047C046F7
:10A6B40030B401256D054C00E54215D85C00E54237
:10A6C40012D80C001C436400044314430CD005D27C
:10A6D400904299418041404230BC704782428B4154
:10A6E4008041404230BC7047002030BC7047C046B7
:10A6F400F4464A1805D200F063F801D5C0174008A3
:10A70400604701235B05D34206D200F059F801D516
:10A714000120C0074042604701D10042F5D0D01764
:04A724004008704732
:10A728004A00520D01239B02D21A01321DD4524213
:10A738003F321DDD8C46C902430D1943C002012377
:10A74800DB071943202A02D308000021203AD1410F
:10A75800D04048409140D140484063461B4203D511
:10A76800002340428B4119007047002000217047A8
:10A77800002801D0012211434B0001225205D34287
:10A7880000D959080020C90FC90701D4C04341089E
:04A798007047C04600
:10A79C0041000DD2090E7F390AD449421F3105D42C
:10A7AC0000020122D2071043C8407047C8177047F7
:04A7BC0000207047C2
:10A7C0004A0010D2520D03231B02FF33D21A0AD4BF
:10A7D00052421F3209D4400DC90208430123DB074E
:10A7E0001843D040704700207047D0177047C046CC
:10A7F0004B001BD25A0D01239B02D21A013215D4F1
:10A8000052423F3215DBC902430D1943C0020123F6
:10A81000DB071943202A02D308000021203AD14146
:10A82000D04048409140D14048407047002000212E
:08A830007047D01701007047CA
:10A83800054B004206D5404200B5984708BC0122A6
:0CA84800D207114318470000D1A80008F7
:10A854000B00034329D0CA0FD200043212023D3246
:10A86400094203D5002349424042994102D10100E3
:10A874000020203A0B0C04D1103A0904030C1943AC
:10A884000004094203D4013A00184941FBD5844627
:10A89400C00A4B051843C90A120563465B055B41B0
:0CA8A40002D3012B0023584151417047A2
:10A8B0009D2201000AD002D4013A4900FCD5D205FC
:10A8C000080A0906494100D3012950417047C04692
:10A8D00042221201033A010007D002D4013A0018C3
:0CA8E000FCD51205C30A4005991870470A
:10A8EC000B00034305D0042212023D320942014BF6
:08A8FC001847704771A800081D
:10A90400202A07D203009040914052422032D34083
:10A9140019437047203A0100914000207047C04617
:10A92400202A07D2D0400B00D1405242203293401B
:10A9340018437047203A0800D04000217047C046B1
:10A94400202A07D2D0400B001141524220329340BA
:10A9540018437047203A08001041C9177047C04691
:10A9640030B5514343435C18010C130C0D005D4397
:10A97400641992B2514380B242430D0C0904521837
:10A9840065415843010C00048018694130BDC0463C
:10A99400CA1751408B1A17D0C1174A4094464840F1
:10A9A400411A48081A0000E052008242FCD90020F3
:10A9B40000E05208914200D3891A40419A42F8D1EA
:10A9C40062465040801A704710B500F095F810BDEB
:10A9D40007B5FFF7DDFF0EBC4243891A00BDC04630
:10A9E4000A0015D00300400800E052008242FCD95E
:10A9F400002000E052089B1A06D340418A42F9D154
:10AA0400704752089B18F8D200188A42F9D170474F
:08AA140010B500F071F810BD4F
:10AA1C0038B504004D42FFF7DFFF4543611938BDDF
:10AA2C0070B5CC1760406140001BA141DD176A4036
:10AA3C006B40521BAB4100F00BF862406340121BA1
:10AA4C00A3416C4060406140001BA14170BDC046F9
:10AA5C00002B09D1002907D110B51100FFF7D8FF41
:10AA6C000A000021002310BD70B400240125ED075D
:10AA7C00002B07D1002905D0834203D213000022FA
:10AA8C002C0000250026A419994200D1904212D91D
:10AA9C0092185B4103D2EE076D086408F3E7DE07FA
:10AAAC005B08520892190126F6079B1903E0DE0792
:10AABC005B0852089219801A994103D364416D4185
:10AACC00F5D30FE024196D410AD2DE075B0852085A
:10AADC00921980185941F5D364416D41E7D301E0D7
:10AAEC008018594102000B002000290070BC7047EF
:08AAFC00002000217047C04654
:10AB0400F0B503AF93B06E46F51D2135F41D39340D
:10AB140074613362F261F160306101F0EAFBB060AC
:10AB2400C21D07218A436946B1616946881A70606B
:10AB34008546F41D1D3400212422204600F0CAFF5E
:10AB44000B487169F2680A6048600A4828603069F5
:10AB54002862B06868617068E8602046F169326A0A
:10AB640000F01EF8B1698D46FE1F053EB546F0BDE6
:08AB7400E7C20008FFFFFF7FAC
:10AB7C0083B010B581B0044603A80EC00548006828
:10AB8C0003AA0092214601F041FA01B010BC02BCAC
:08AB9C0003B00847140000207B
:10ABA400F0B59FB012920B460446002020600121AC
:10ABB4000A020F924A020B928A020192CA0200927E
:10ABC40003220D92920205920D034A0307928A030F
:10ABD40003920491C90317910A90C04302901694FA
:10ABE40009951978252909D0002901D100F03CFEE6
:10ABF4005C1C169801F0B1F92346F2E7DB1C0A9FAE
:10AC04000B9C981E00780246203A102A2CD88021EA
:10AC140092003E461F4602A39A583B463746974643
:10AC240069AC000889AC000889AC000883AC000852
:10AC340089AC000889AC000889AC00087DAC000828
:10AC440089AC000889AC0008ADAC000881AC0008F0
:10AC540089AC000875AC000889AC000889AC000810
:10AC640079AC000840210AE05E28294607D009E0B3
:10AC7400102104E0214602E0179900E020210F434F
:10AC84005B1CBEE75B1E014630390024092916D837
:10AC94000A2161434418303C591C18780246303A62
:10ACA4000A2A0B46F4D30AE0129901C91291C10F82
:10ACB40009010F43C1174840441A581E0078002662
:10ACC4002E281CD118782A2805D158789B1C129953
:10ACD40040C912910FE05B1C0146303909290CD898
:10ACE4000A2171434618303E591C18780246303AFE
:10ACF4000A2A0B46F4D3002E01D40F990F43E1170F
:10AD04006B2808DC4C2803D068283CD06A280AD178
:10AD14000220074305E06C2830D07A2801D074283B
:10AD240001D118785B1C8C43462811931BDD014626
:10AD34006339152937D8C0467944097949008F44C5
:10AD4400710B4D1BD70A0B0A0A0A0A8194610A0A7D
:10AD54008F0A560A0A3A44E70C94039C27430021BD
:10AD6400089139468EE0442815DD452834D046281C
:10AD740000D036E7079807430098BAE018786C28A3
:10AD84002ED1022003E0187868282CD1082007432C
:10AD940058789B1CC7E7252800D08EE225211698F9
:10ADA40001F0DBF87AE2472800D19FE0582800D070
:10ADB40017E707990F430C94D34A782800D120321F
:10ADC400039C0F990F42394601D0D04B19403B06E2
:10ADD400DB171340089355E007980743019888E070
:10ADE4005B1C049A01E05B1C042217439BE70C9450
:10ADF4000F990F4201D0C5490F403946039C0022E8
:10AE040008923FE00C9438060F990F430E97C01731
:10AE1400232101400891129820C812900024082090
:10AE24000690D3E1129E3578621E169C2046394660
:10AE3400159201F0E4F82046294601F08EF8361DFB
:10AE44001296C2E01298006839071699096800D56D
:10AE540037E2BA07016000D434E20021416031E2F4
:10AE64001596129901C912918EE00C940F990F4214
:10AE7400394601D0A54A11403A06D217302313406F
:10AE84000893039C02220A40214205D1002A129A07
:10AE940008D1131D00240BE0002A129B13D104CB0C
:10AEA400D41715E0D21D07239A4354681346083378
:10AEB400129315684A0713D408220A4000D0EDB251
:10AEC400002A0ED102E1DB1D0722934314CB003389
:10AED40012934B0707D40B0700D5E3E01546E4E0D3
:10AEE400ADB20024F2E015B21204DDE00798074386
:10AEF400059807430F98074201D0304600E006202A
:10AF04000C943946059A1140891A4A424A4100284C
:10AF140000D002461592129CE41D07208443266843
:10AF2400656830462946FEF721FD0834129400284E
:10AF3400304629460ED000221346FFF7B9FB3A46A5
:10AF440007990A4000280C9C0FD0002A704819D099
:10AF5400704817E0FEF7FCFC00280C9C37D00798DB
:10AF640007426D480ED06D480CE0002A6C4900D0B1
:10AF74006C49002A01D06B4800E06948401CBA06BD
:10AF840000D5084668490F400028684E00D00646A0
:10AF94000F980742304602D100F016FD02E01599E1
:10AFA40000F04AFD054659480740621B1698394689
:10AFB400159201F024F8002D07D0169C3178204614
:10AFC40000F0CBFF761C6D1EF8D1F8065DE130462B
:10AFD4002946FEF7D7FC002800D10646002800D1F8
:10AFE400002513963046294601F017F9044601203E
:10AFF400002C089001D0C00745401EAA3046109589
:10B004002946FEF7F7FC1E980D9948430A21FFF7DD
:10B01400BFFC06461E90002C01D06020074300228E
:10B02400139C2046294614921346FFF7E7FA00289A
:10B0340018D1701CFFF7E8F822462B46FFF738FBBF
:10B0440000281E9806D0411C1E91801CF2E71E9811
:10B05400401E1E90FFF7D8F822462B46FFF708FB48
:10B064000028F4D13D4605980540089883021E98AF
:10B074009D42159E00D113E105998D4207D1864268
:10B0840000DC0DE10421C943884200DC08E1019998
:10B094000F42109D0E9300D180E20E2800DCD0E117
:10B0A400149E7BE255B21206D417002C05D48A06EE
:10B0B4000AD44A060AD5202207E000226D42A241A2
:10B0C4002D230893144601E02B2208920F9A114273
:10B0D40001D00E4A11400A460F990E920A42049971
:10B0E40000D03146069100276E2838DD6F380928D4
:10B0F40000D98AE07844007940008744196786863D
:10B10400868636868667C04658300000FFFDFFFFFE
:10B1140007C9000802C900081CCB000818CB0008A6
:10B1240011C900080CC90008FFFEFFFF20C5000874
:10B134002846204369D0E8086107401801460720E3
:10B144002840303018AAD055C808E408620780188F
:10B154000A4622437F1C002A0D46EFD155E05828A9
:10B1640034D0642801D069284FD1284620434CD0DC
:10B1740011461798014010912A461098002808D0CB
:10B1840038460D990840032803D118A82C21C1552D
:10B194007F1C002510462146159414460A222B468E
:10B1A400FFF75AFC149013910A222B46FFF7D8FBA1
:10B1B400201A3021014318A8C1557F1C0920001B07
:10B1C40015988541149D139CD6D31EE02846204330
:10B1D4001AD007980E990142C04800D0C0482909E6
:10B1E4002207891800270A460F212940415C18AB21
:10B1F400D955110924092307C918134623437F1C71
:10B20400002B1546EFD100E00027089DFF2D01D843
:10B21400029801E0B348FF300B9C0C9B0699CE1BAF
:10B22400F1178E43B9195A1A002D00D012180E992D
:10B23400214203D1169800F0E2FE00221592290A59
:10B24400169C03D0204600F088FE01E0002D03D0B8
:10B254002046294600F081FE20460E99159A00F0FA
:10B26400CEFE30212046324601F02DF8012F0ADBB4
:10B274007D1C18A84019801E0178204600F06DFE40
:10B284006D1E012DF5D80E98C006099D119B00D4A2
:10B29400A7E420211698159A01F015F8119BA0E453
:10B2A4000F9934318842109C06950FD1139821468A
:10B2B4008D4A8E4BFFF71EF90FE0002800D090E472
:10B2C400E2E201701298001D12908AE44042FEF7F7
:10B2D4009BFF139A234600F097FD04460E46002276
:10B2E4001346FFF78BF9002839D120463146FEF783
:10B2F4003DFB00282046314600D01CE60E97002274
:10B304007B4BFFF793F900281E9F0FD000222046A5
:10B314003146774BFFF7EEF804460E460022744B95
:10B32400FFF784F97F1C0028F0D11E9700222046E5
:10B334003146704BFFF7BCF9002811D0002220469B
:10B3440031466B4B00F060FD04460E460022694B0B
:10B35400FFF7AEF97F1E0028F0D11E9700E00E978C
:10B36400059806998142159801D0014600E0411ED6
:10B37400029D0028149100D1002113914842FEF748
:10B3840043FF2A46FEF712FB22463346FEF76AFFC6
:10B3940006460D4600220692554C2346FFF746F911
:10B3A40000280AD01E98401C1E90002230462946D0
:10B3B4002346FFF79FF806460D46109615951398F9
:10B3C400002866D000990B4680330E9A13408B42B6
:10B3D40061D1102800DB10200546FEF715FF324628
:10B3E400159B00F011FDFFF701FA0C4601462143BD
:10B3F400069914914FD0214606463F4A3F4BFFF72A
:10B40400AFFA4A08C3079A184008C90708183C4904
:10B41400081A3C48904114953DD330460A22002333
:10B424002146FFF719FB0C4607460A220023FFF7C3
:10B4340013FB1498401E14902DD01A433846EDD0B7
:10B4440029E0C143711810290E4600DB10263A0684
:10B4540000D5A3E0002900D1A0E03046FEF7D4FED9
:10B46400139A2B4600F0D0FC00242246264BFEF70C
:10B47400F9FEFEF799FB22461D4BFEF7D7FA22464A
:10B484002346FFF7BBF8002800D184E0761EE4D100
:10B4940082E00698149080210E9806460140149A82
:10B4A40011430C98801A002901D1401F00E0801F2D
:10B4B400139009981E9C064201D1089D46E0032181
:10B4C4002046FFF785FA881C0125C0467844007998
:10B4D400400087441B2A381B2A00C04608CB0008BA
:10B4E400F8CA0008FFFEFFFFA0C8EB85F3CCE17F9C
:10B4F400000024400000F03FCDCCCCCCCCCCCCCC54
:10B5040099999999999999190000E03F641E1E949C
:10B51400002210981599DF4B00F076FC10901591DD
:10B524001398401E139002250DE0A41E1E940022C1
:10B5340010981599D84B00F067FC1090159113984A
:10B54400801E13900325149AD01782437006800F2F
:10B55400149202D01398401E1390204600F0AFFEC0
:10B56400632802DD1398401E13900898C0023746E2
:10B57400874310981599FFF739F906460C46FFF7EB
:10B58400B3F902460B4610981599FEF74FFF109039
:10B594001591139A76E034461E9826461038149670
:10B5A4007142884200DC0846FEF72EFE029AFEF73E
:10B5B400FDF9139A2B46FEF755FE05460C461E98D8
:10B5C400401CFEF721FE2A462346FEF7F5FF00281D
:10B5D4001E9800D0401C002814D4112818D301460A
:10B5E40010391E911021081AFEF70EFE2A46234632
:10B5F40000F00AFCFFF7FAF806460C460020159006
:10B60400109018E01095159400261E96344612E00A
:10B6140000201E9028462146FFF7E8F806461594B8
:10B624000C46FFF761F902460B4628461599FEF7CA
:10B63400FDFE1090159138460E99884397490831BC
:10B6440000250A4608326D1C0B684968F31A234624
:10B654008B411146F6D280213940149A11434B1E76
:10B664000A469A41002901D00021C9437B069B0F59
:10B6740000D0D1431E9A891A0C9A149BD21A5118DD
:10B684004A1B0746D017114681430B9810300E977A
:10B6940007420AD1012A08DB0F462021169800F040
:10B6A4005CFC7F1EF9D10E9A01E03A460F46402019
:10B6B4001040910603D4002809D0202104E000287A
:10B6C40001D02D2100E02B21169800F046FC0E98A5
:10B6D400C00607D4002F05D03021169800F03DFC99
:10B6E4007F1EF9D16D1EE8006C4A11184968125882
:10B6F400B01A2046884101D2302007E03020B61A23
:10B704008C41401CB31A23468B41F8D2C1B216981F
:10B7140000F023FC002DE5D113970E9E34460098CB
:10B724000440169F0BD01E98012808DB401E1E9073
:10B734003021384600F011FC1E980028F6DC8020E9
:10B7440030401499084344D02E21384600F005FCBB
:10B75400149D102D00DB1025E8178543002C01D122
:10B76400284601E01E98281A159CFEF74DFD149AF0
:10B77400012A22DB109A234600F046FBFFF736F835
:10B7840004460E462F467F1EF800444A11184968A5
:10B794001258A01A3046884101D2302007E03020E8
:10B7A400A41A8E41401CA31A33468B41F8D2C1B26D
:10B7B400169800F0D2FB002FE5D11499481B169F70
:10B7C4000E9E06D06C1A3021384600F0C6FB641C6D
:10B7D400F9D301980642099D139F38D00798064271
:10B7E40001D0452100E06521169E304600F0B5FBEE
:10B7F4001E980028304604D42B2100F0AEFB1E987E
:10B8040005E02D2100F0A9FB1E9840421E906428FB
:10B814000DDB6421FFF7E4F801463031304600F0D7
:10B824009CFB1E986421FFF7D3F808461E910A2159
:10B83400FFF7AEF801463031304600F08EFB1E981B
:10B844000A21FFF7C5F83031304600F086FB002F9F
:10B85400119B01D1FFF7C5F9169C2021204600F069
:10B864007CFB7F1EF9D119E5169CE068002805D001
:10B8740006CC083C914201D20A9A4254204600F078
:10B88400B1FB20681FB0F0BD169800F0ABFB029826
:10B89400F8E7C04600002440000059403001000889
:10B8A40009490968091A4A1E9141084A1268121A7C
:10B8B400531E9A410A4006490968081A411E8841E4
:10B8C400104040427047C046140000201800002079
:04B8D4001C00002034
:10B8D8000F480321016141610E4A82610E49C1612D
:10B8E800012189020162002181624162C16202660E
:10B8F8000A4A4266102282660167C1664167084AA1
:10B908000F234B40D35C4354491C1029F8D170478E
:10B91800EC09002027C90008950F00209513002086
:04B9280016C9000834
:10B92C00F0B581B00D461821414316484618F06A0F
:10B93C00183602281ED0144601280ED000270028E5
:10B94C001DD1304600F074FBA04218D33046294676
:10B95C00224600F078FB274611E0304600F068FBE9
:10B96C000746A04200D32746304629463A4600F007
:10B97C006AFB04E03046294600F082FB0746384655
:08B98C0001B0F0BDEC09002040
:10B99400F0B581B014460D4606460A4800780028E2
:10B9A40001D1FFF797FFEFF31087012181F310888E
:10B9B400304629462246FFF7B7FF87F3108801B0C7
:08B9C400F0BDC046EC090020B3
:10B9CC00F0B581B00178002925D003220146009200
:10B9DC0091430D680023DC438607F60EB440E44324
:10B9EC002C43114D6719A743104A174206D14C68D6
:10B9FC0067191646A643091D3E42F8D022060FD001
:10BA0C002204120E09D02202120E08D0220E009B24
:10BA1C0006D0042304E0002004E0012300E002230C
:10BA2C00C918081A01B0F0BDFFFEFEFE80808080B0
:10BA3C00F0B581B00022002934D00378002B31D02E
:10BA4C0003270246BA430024E5438607F60EB540A9
:10BA5C00EE431568354306463E40711804290CD355
:10BA6C000097134EAF19114BAB433B4204D1091F46
:10BA7C005568121D0329F5D8009F2B060DD02B04F9
:10BA8C001B0E07D02B021B0E06D02B0E00D004274A
:10BA9C003C4602E0012400E002248C4200D30C4618
:10BAAC00101A0219104601B0F0BDC046808080808B
:04BABC00FFFEFEFE8D
:10BAC000002A03D0013A8B5C8354FBD17047C046F7
:10BAD00000220B0011001A00002A02D0013A815402
:04BAE000FCD17047DE
:10BAE400002A09D0884207D007D280188918524208
:10BAF4008B5C83540132FBD17047013A8B5C8354D5
:04BB0400FBD17047BA
:10BB080002480068002800D1014870471C0F002037
:04BB18000000002009
:10BB1C007F2805D8034A125C0348405C10407047EC
:0CBB2C000020704720CB000891C90008E1
:10BB38007F2805D8034A125C0348405C10407047D0
:0CBB48000020704720CB000891C90008C5
:10BB540000000000040000000200000008000000D3
:10BB640001000000020000000400000006000000C4
:10BB7400080000000A0000000C0000001000000093
:0CBB8400200000004000000080000000D5
:10BB900000000000000000000000000000000000A5
:10BBA0000000000000000000000000000000000095
:10BBB000010000000200000003000000040000007B
:10BBC0000600000007000000080000000900000057
:10BBD0000000000000000000000000000000000065
:10BBE000010000000200000003000000040000004B
:0CBBF000FEC600081CBC0008FCBB0008DE
:10BBFC001DBB00080BC3000819C1000839BB0008A5
:10BC0C0017C3000827C10008FBC20008EBC00008DE
:10BC1C0000C7000890C9000890C9000890C9000826
:10BC2C0090C9000890C9000890C9000890C9000884
:10BC3C0090C9000890C90008FFFFFFFFFFFFFFFF3E
:10BC4C00FFFFFFFFFFFF0000C4C6000842C9000849
:10BC5C0027C500085FC900087EC5000830C9000868
:08BC6C0039C9000885C5000874
:10BC7400034C206804348047FBE7F7F7B1FEFEE786
:04BC8400A0CB000849
:10BC880004480549884385460448804704480549CF
:10BC98000160EBE70080002007000000B1BD00084C
:08BCA80008ED00E000000008B7
:10BCB000FEE7FEE7FEE7FEE7FEE7FEE7FEE7FEE75C
:10BCC000FEE7FEE7FEE7FEE7FEE7FEE7FEE7FEE74C
:10BCD000FEE7FEE7FEE7FEE7FEE7FEE7FEE7FEE73C
:10BCE000FEE7FEE7FEE7FEE7FEE7FEE7FEE7FEE72C
:0CBCF000FEE7FEE7FEE7FEE7FEE7FEE7EA
:02BCFC0070478F
:10BCFE0030B580214158212918D102465632938AF7
:10BD0E00002B13D0016802E05B1E1C040ED01488B9
:10BD1E00002C0CD0CC692406F6D5046D25788D62E6
:10BD2E00641C04651488641E1480EDE730BD012088
:10BD3E00C0058A6882438A600868402202430A600E
:02BD4E0030BD06
:10BD500010B5842141582229016810D102465E3273
:10BD60005388496A1940836D19701188491E1180E2
:10BD7000816D491C81651188002905D010BD886935
:10BD8000082202438A6110BD014684310922520112
:10BD900003681C6894431C609A680124A2439A605B
:0ABDA0000022C2662020086010BDDA
:02BDAA007047E0
:02BDAC007047DE
:02BDAE007047DC
:02BDB0007047DA
:10BDB20010B582B00B4601AC2070012120460A4624
:10BDC20000F012FA002801D0207800E0C04302B04F
:02BDD20010BDA2
:10BDD40008D1002806D1F54204D801D3002A01D1A4
:10BDE4006D0D09D10020C143090DC904F0BDF9D17D
:10BDF4001242F7D1640DF5D00020C143490549082A
:10BE0400A6E000206146F0BDF0B50127FF070E0053
:10BE14005E403E40B446BE0A4C18DD18F442D7D208
:10BE2400F542E4D2640DECD06D0DEAD06419C90278
:10BE34003943460DC0023143DB023B43DB0A10B4F5
:10BE44008E4685B297B26F43140C6C433E0CA41912
:10BE5400260C2404BFB227439CB26C43A419190CCA
:10BE64006943250CA4B249190D04090C6419000C8A
:10BE740095B245433E0C76193743BFB2360C150CC8
:10BE84004543AD19A6B2240CAD192E0437432E0C2C
:10BE940036199DB24543AD19ACB22E0C89191D0C4F
:10BEA40045436D182E04290C3443704680B295B274
:10BEB40045433E0C76193743BFB2360C150C454347
:10BEC400AD19A6B2AD19240C2E0437432E0C361925
:10BED4009DB24543AD19ACB22E0C89191D0C4543D6
:10BEE4006D182E043443290C75462D0C90B268430A
:10BEF4003E0C80190604BFB23E43070CA0B23F18A3
:10BF0400120C6A43D019020C80B2240CA4189AB201
:10BF14006A43121914042043120C89181B0C6B4336
:10BF2400C91810BC01273D05294203D1B619404167
:10BF34004941013CFF077D0D013D641B0BDB6D0096
:10BF4400AC4209DA240500254208BE41684161413A
:0ABF540066463143F0BD54E74EE7A6
:10BF5E0030B581B0044668460170206900280FD0C4
:10BF6E000CCC083C9A4233D26269531C63618154F3
:10BF7E00A069616981422BD1204600F02EF827E09E
:10BF8E00E068002809D00CCC083C9A4220D2551CFF
:10BF9E009D4200D1002181541AE0A068002808D0EB
:10BFAE000CCC083C9A4213D2551C9D420DD0C9B2FE
:10BFBE000CE0236A002B0BD003CC083C884207D23E
:10BFCE00694601222046984702E0002192008150E6
:0ABFDE002068401C206001B030BD57
:10BFE80010B54269002A07D00446036A002B01D025
:0ABFF800216998470020606110BD28
:10C0020080B5CB0606D4890501D5302100E0202178
:06C0120000F05AF980BDA8
:10C0180070B514460D460646FFF772FD01463046D8
:0AC028002A462346FEF76AFD70BDAC
:0AC0320080B50068FFF7ADFC80BD8B
:10C03C00C2680169914201D9D04302E0D243891808
:06C04C008068081870472F
:10C05200F0B581B0154604464068A268E6688019CA
:10C06200971BBD4204D22A46FFF729FD751909E044
:10C072000E463A46FFF723FDF119ED1B60682A468A
:0AC08200FFF71DFDE56001B0F0BD01
:10C08C00F0B583B016460D46C768002101900291A9
:10C09C000269F943BA4202D95418816802E0521875
:10C0AC00816854184268C91B8C4200D30C46B442B8
:10C0BC0000D33446D01929462246FFF7FBFCE7197A
:10C0CC00019881688F4200D100270299C760361B06
:0EC0DC002D196118002EDAD1084603B0F0BD10
:10C0EA0010B50446002000290DD0002A0BD009788B
:10C0FA0048B2002808D4002C00D021600021196021
:0EC10A005960411E884110BD0120C04310BD88
:0EC11800014641391A2901D2202108437047FF
:0EC12600014641391A2901D2202108437047F1
:10C13400010002000400060008000A000C001000C0
:06C1440020004000800015
:10C14A00806A816D40220A438265C16D04220A43D6
:04C15A00C265704703
:10C15E0010B580214258212A0DD1034656331A8834
:10C16E00002A026808D0016D0C789462491C0165A2
:10C17E001888401E188010BD106888431060106823
:08C18E0040210143116010BDC6
:10C1960010B584214158222901680FD102465E322A
:10C1A60053884C6A1C40836D1C801488641E14805E
:10C1B6009B1C83651288002A05D010BD8869082259
:10C1C60002438A6110BD092252010B6893430B603A
:10C1D6008A6801239A438A600021C166843020213F
:04C1E600016010BD27
:10C1EA00F0B581B01E4615460C4607461846FFF7BD
:10C1FA0054FB0146002000290AD46543A54207D30F
:10C20A00304639462A46FFF70FFF2146FEF7E5FB7F
:04C21A0001B0F0BDC2
:04C21E00C80F70478E
:10C22200F0B581B01C4615460091CA0017183E466B
:10C23200103EB068F1682A46FFF7E7FD0CCEFEF724
:10C2420012F8009A032A0DDB183F561E2A4623468F
:10C25200FFF7DBFD0CCF083FFEF705F8761E083F1F
:10C26200012EF3D82A462346FFF7CFFD01B0F0BDD9
:10C27200F0B581B01D4616460346C800022916DBFA
:10C2820000931F18083F4C1C304629460CCF083F2C
:10C29200FDF7E9FF32462B46FFF7B7FD641E083F64
:10C2A200022CF3D8009B083306460D4600E01B180B
:10C2B200083B0CCB30462946FDF7D5FF01B0F0BD57
:08C2C200C1174840401A704703
:10C2CA0070B5012A09DB0C460546561C284621464C
:0CC2DA00FFF740FE761E012EF8D870BD64
:10C2E60010B50C46436A01212046FFF77BFF10BDBF
:04C2F600402070472D
:10C2FA00024601207F2901D9C04370471170704757
:0CC30A00014661391A2900D22038704722
:0CC31600014661391A2900D22038704716
:0FC3220049205265666572656E7A3D25660A0090
:0BC33100547368756E743D25660A00A9
:10C33C002D2D2D204761696E20447269667420434F
:07C34C00414C202D2D2D00B6
:0FC3530041637475616C20543D256620430A00D8
:10C3620041637574616C20493D25662041287769D7
:10C3720074686F7574206761696E2074656D7020D2
:10C38200647269667420636F7272656374696F6E3A
:03C39200290A0075
:10C395004B6F7272656B74757266616B746F723D0B
:10C3A5002566205B2031202F2043656C73697573EA
:03C3B5005D0A001E
:10C3B8004552524F52204144535F313236305F5319
:0BC3C80065744461746152617465008B
:10C3D3004552524F52204144535F313236305F53FE
:0BC3E300657443686F704D6F64650067
:10C3EE00454550524F4D20776173206368616E67EB
:10C3FE00656421205765206E65656420746F20701A
:10C40E00726573657276652063616C6962726174C0
:10C41E00696F6E20616E642073657474696E6773E4
:07C42E00206461746121002C
:10C43500454550524F4D20464143544F5259205285
:0FC445004553544F52452F555044415445210003
:0FC454007265616420636F6E6669672E2E2E001D
:10C46300666163746F727920726573746F72652E7F
:03C473002E2E006A
:10C4760050524F54454354494F4E3A204F425F5213
:0BC4860044505F4C4556454C5F3200AF
:10C4910050524F54454354494F4E3A204F425F52F8
:0BC4A10044505F4C4556454C5F310095
:10C4AC0050524F54454354494F4E3A204F425F52DD
:0BC4BC0044505F4C4556454C5F30007B
:10C4C700466C61736820756E6C6F636B2065727262
:03C4D7006F720081
:10C4DA004F5554505554535F4C56505F5348554E20
:10C4EA00545F554E44455254454D5045524154555A
:03C4FA00524500A8
:10C4FD004F5554505554535F4F56505F5348554EFA
:10C50D00545F554E44455254454D50455241545536
:03C51D0052450084
:07C52000286E756C6C290008
:10C527004A616E75617279004665627275617279EA
:10C53700004D6172636800417072696C004D6179EA
:10C54700004A756E65004A756C79004175677573A9
:10C55700740053657074656D626572004F63746F24
:10C56700626572004E6F76656D6265720044656341
:07C57700656D6265720000B2
:07C57E00414D00504D00008B
:0FC5850025612025622025652025542025590099
:0EC5940075617274206572726F72200A0D005C
:10C5A2002D2D2D204761696E202043414C202D2DD9
:02C5B2002D005A
:0AC5B40054736869703D25660A00A3
:10C5BE002D2D2D204761696E202043414C20454E84
:06C5CE0044452D2D2D0057
:0EC5D40064656C746120543D256620430A00A6
:0AC5E20052656620493D25660A00F7
:10C5EC004552524F52204144535F313236305F49ED
:0EC5FC006E7075744D757853656C65637400D0
:10C60A004669727374207374617274206465746508
:06C61A0063746564210059
:0EC620004953454E534F523A20496E697400FB
:10C62E002E2E2E466C61736820756E6C6F636B6573
:02C63E00640096
:10C64000466C617368206F6220756E6C6F636B203F
:06C650006572726F7200BA
:0EC65600466C61736820206C6F636B65640036
:10C664004F5554505554535F4C56505F5348554E94
:10C67400545F4F56455254454D50455241545552BE
:02C6840045006F
:0EC686004F5554505554204C5650204F4B00E9
:10C694004F5554505554535F4F56505F5348554E61
:10C6A400545F4F56455254454D504552415455528E
:02C6B40045003F
:0EC6B6004F5554505554204F5650204F4B00B6
:10C6C40053756E646179004D6F6E646179005475C1
:10C6D4006573646179005765646E6573646179009C
:10C6E4005468757273646179004672696461790093
:0AC6F40053617475726461790000EF
:02C6FE004300F7
:02C700002E0009
:10C702004672657175656E6379204D6561737572E8
:09C712006564203D2025640A0045
:10C71B00492028776974686F757420636F6D706535
:0DC72B006E736174696F6E293D25660A000A
:10C738004144535F313236305F42617474657279B7
:10C7480043757272656E744761696E43616C6962A4
:10C75800726174696F6E53746172743A20455252F3
:10C768004F5220494E2043414C4942524154494F6F
:10C778004E2C204E4F205245464552454E434520AB
:09C7880043555252454E54210064
:10C791004E6F726D616C207374617274207769746D
:10C7A100686F757420454550524F4D206368616E26
:0DC7B10067657320646574656374656400DA
:10C7BE00454550524F4D2046554C4C2052455354F2
:05C7CE004F524521005F
:10C7D300454550524F4D2053544F524520434F4EE1
:05C7E30046494721005A
:0DC7E8004144533132363020496E697400EF
:10C7F5002E2E2E466C617368206F6220756E6C6FED
:05C80500636B65640097
:10C80A002E2E2E44697361626C65206C6F636B20F7
:10C81A0070726F636573732066696E6973686564A5
:01C82A00000D
:10C82B00466C617368204F7074696F6E62797465C2
:10C83B002070726F6772616D6D206661696C6564E3
:01C84B0000EC
:10C84C002E2E2E466C617368206C6F636B20616CAE
:0DC85C00726561647920616374697665001E
:10C869002E2E2E456E61626C65206C6F636B2065A0
:05C8790072726F7200F5
:10C87E004F5554505554535F4C56505F4348495092
:10C88E005F4F56455254454D5045524154555245B1
:01C89E000099
:10C89F004F5554505554535F4C56505F424154546A
:10C8AF004552595F554E444552564F4C544147459A
:01C8BF000078
:10C8C0004F5554505554535F4F56505F434849504D
:10C8D0005F554E444554454D50455241545552457F
:01C8E0000057
:10C8E1004F5554505554535F4F56505F434849502C
:10C8F1005F4F56455254454D50455241545552454E
:01C901000035
:05C902002D494E460026
:05C907002D696E6600C1
:05C90C002B494E46001E
:05C911002B696E6600B9
:10C91600000000000000545452205245474745533A
:01C926000010
:09C927005465726D696E616C00CB
:09C93000256D2F25642F257900E7
:09C9390025483A254D3A2553002A
:10C9420053756E004D6F6E00547565005765640037
:0DC95200546875004672690053617400005E
:10C95F004A616E00466562004D617200417072005F
:10C96F004D6179004A756E004A756C00417567001C
:10C97F00536570004F6374004E6F7600446563001B
:01C98F0000A7
:01C9900000A6
:0DC991000007032004170201085710408022
:04C9A000899800086A
:10C9A40056616C7565206E6F742076616C696400E5
:10C9B4004B6F7272656B74757266616B746F723DE6
:04C9C40025660A00DA
:10C9C8002D2D2D204761696E2044726966742043BD
:0CC9D800414C20454E4445202D2D2D00E3
:10C9E4004552524F52204144535F313236305F53E7
:10C9F4006574496E7465726E616C526566657265C4
:04CA04006E636500F8
:0CCA080057726974696E6720534E21005C
:10CA1400554E4B4E4F574E20434F4D4D414E4400C3
:10CA2400466C617368204F7074696F6E62797465C7
:0CCA34002070726F6772616D6D656400A8
:10CA4000537461727420656E61626C6520726561F9
:10CA5000646F75742070726F74656374696F6E00B3
:10CA60002E2E2E466C61736820756E6C6F636B00A2
:10CA7000466C617368204F7074696F6E627974657B
:08CA8000206C6F636B6564001C
:10CA88002E2E2E456E61626C65206C6F636B207074
:10CA9800726F636573732066696E69736865640095
:10CAA8004F5554505554535F4C56505F4F5645524E
:08CAB80043555252454E540053
:10CAC0004F5554505554535F4F56505F4F56455233
:08CAD00043555252454E54003B
:10CAD8004F5554505554535F4F56505F424154542C
:10CAE8004552595F4F564552564F4C5441474500A1
:10CAF800303132333435363738394142434445468C
:10CB080030313233343536373839616263646566BB
:04CB18004E414E003C
:04CB1C006E616E00D8
:10CB2000202020202020202020682828282820209D
:10CB300020202020202020202020202020202020F5
:10CB400048101010101010101010101010101010AD
:10CB5000848484848484848484841010101010104D
:10CB600010818181818181010101010101010101A6
:10CB7000010101010101010101010110101010105A
:10CB80001082828282828202020202020202020277
:10CB9000020202020202020202020210101010201F
:10CBA00015CC000824000020610F000015CC0008FF
:10CBB000860F00200300000015CC00088A0F00201B
:10CBC0000300000015CC00088E0F002003000000B9
:10CBD00015CC0008920F00201304000027CC000899
:10CBE00000000020F0CB0008240000007FBC0008FB
:10CBF000F0BB0008F0BB0008F0BB0008F0BB000869
:10CC0000F0BB0008100F0020140F0020180F0020A8
:04CC10000024F40008
:10CC1400206861680834002200E042540139FCD5E0
:02CC2400704757
:10CC260020686168A2680C3401E08B5C8354013A89
:04CC3600FBD5704773
:020000040801F1
:04C7FC001F4DDADB18
:040000050800BC89AA
:00000001FF
